:020000040000FA
:0408000027EF08F0E6
:1008100003B213EF05F0F2B42EEF05F09EB036EF01
:1008200005F09EB23EEF05F0F2A81AEF04F0F2B226
:1008300025EF04F0F2A620EF04F0F2B022EF04F06E
:10084000D6EF07F0F296F290FF00CD90F2929EA0C4
:100850002FEF04F00101533F2FEF04F0542BAEC1F2
:10086000B2F1AFC1B3F1B0C1B4F1B1C1B5F1AAC138
:10087000AEF1ABC1AFF1ACC1B0F1ADC1B1F1A6C148
:10088000AAF1A7C1ABF1A8C1ACF1A9C1ADF1A2C158
:10089000A6F1A3C1A7F1A4C1A8F1A5C1A9F19EC168
:1008A000A2F19FC1A3F1A0C1A4F1A1C1A5F19AC178
:1008B0009EF19BC19FF19CC1A0F19DC1A1F196C188
:1008C0009AF197C19BF198C19CF199C19DF1CECF4E
:1008D00096F1CFCF97F153C198F154C199F1CF6AF6
:1008E000CE6A0101536B546B9E90CD800FBC0F8E6E
:1008F0000FBA7EEF04F00F8AD6EF07F00F8C0FBE11
:10090000BAEF04F096C19AF197C19BF198C19CF19E
:1009100099C19DF19AC19EF19BC19FF19CC1A0F12B
:100920009DC1A1F19EC1A2F19FC1A3F1A0C1A4F1FB
:10093000A1C1A5F1A2C1A6F1A3C1A7F1A4C1A8F1CB
:10094000A5C1A9F1A6C1AAF1A7C1ABF1A8C1ACF19B
:10095000A9C1ADF1AAC1AEF1ABC1AFF1ACC1B0F16B
:10096000ADC1B1F1AEC1B2F1AFC1B3F1B0C1B4F13B
:10097000B1C1B5F101015E6B5F6B606B616B96514C
:100980005E2797515F2398516023995161239A51B3
:100990005E279B515F239C5160239D5161239E5193
:1009A0005E279F515F23A0516023A1516123A25173
:1009B0005E27A3515F23A4516023A5516123A65153
:1009C0005E27A7515F23A8516023A9516123AA5133
:1009D0005E27AB515F23AC516023AD516123AE5113
:1009E0005E27AF515F23B0516023B1516123B251F3
:1009F0005E27B3515F23B4516023B5516123D89072
:100A00000101613360335F335E33D890010161339C
:100A100060335F335E33D8900101613360335F33FD
:100A20005E33D6EF07F00392030103EE00F080512E
:100A30007F0BE92604C0EFFF802B8151805D700B96
:100A4000D8A48B8200008051815D700BD8A48B925A
:100A500081518019D8B40790D6EF07F0F2940101C4
:100A6000453FD6EF07F0462BD6EF07F09E900101E9
:100A7000533FD6EF07F0542BD6EF07F09E920400B9
:100A800062A143EF05F007B495EF05F007B095EFCD
:100A900005F01EC620F61FC621F61CC61EF61DC692
:100AA0001FF61AC61CF61BC61DF606C608F607C6B4
:100AB00009F604C606F605C607F602C604F603C61E
:100AC00005F626C628F627C629F624C626F625C624
:100AD00027F622C624F623C625F60EC610F60FC644
:100AE00011F60CC60EF60DC60FF60AC60CF60BC6AE
:100AF0000DF62EC630F62FC631F62CC62EF62DC6B4
:100B00002FF62AC62CF62BC62DF616C618F617C6D3
:100B100019F614C616F615C617F612C614F613C63D
:100B200015F693EC2AF02BEC2AF0077C07ACB0EF1B
:100B300005F0C274C2B4AAEF05F0C3CFB3F5C4CFB9
:100B4000B4F50501D890B433B333D890B433B3338C
:100B5000B1EF05F0C3CF55F1C4CF56F1B1EF05F0B9
:100B6000C28207B41EEF06F047C14BF148C14CF1F9
:100B700049C14DF14AC14EF15EC162F15FC163F1FD
:100B800060C164F161C165F196C1B6F197C1B7F179
:100B900098C1B8F199C1B9F19AC1BAF19BC1BBF141
:100BA0009CC1BCF19DC1BDF19EC1BEF19FC1BFF111
:100BB000A0C1C0F1A1C1C1F1A2C1C2F1A3C1C3F1E1
:100BC000A4C1C4F1A5C1C5F1A6C1C6F1A7C1C7F1B1
:100BD000A8C1C8F1A9C1C9F1AAC1CAF1ABC1CBF181
:100BE000ACC1CCF1ADC1CDF1AEC1CEF1AFC1CFF151
:100BF000B0C1D0F1B1C1D1F1B2C1D2F1B3C1D3F121
:100C0000B4C1D4F1B5C1D5F1B3C5B5F5B4C5B6F528
:100C1000B5C5B7F5B6C5B8F5010155515B275651B5
:100C20005C23E86A5D230E2E1EEF06F05CC157F1CF
:100C30005DC158F15B6B5C6B5D6B078E0201002F31
:100C4000D6EF07F03C0E006F05012F51000AD8B413
:100C5000D5EF06F005012F51010AD8B45FEF06F079
:100C600005012F51020AD8B4A0EF06F005012F515B
:100C7000030AD8B4A0EF06F005012F51040AD8B436
:100C8000A0EF06F005012F51050AD8B4A0EF06F039
:100C900005012F51060AD8B4A0EF06F005012F5127
:100CA000070AD8B4A0EF06F005012F51320AD8B4D4
:100CB0005DEF06F02F6BD5EF06F0D5EF06F00501DE
:100CC00053676AEF06F054676AEF06F055676AEFFC
:100CD00006F056676EEF06F0D5EF06F057C500F147
:100CE00058C501F159C502F15AC503F10101010EC0
:100CF000046F000E056F000E066F000E076F9CEC70
:100D000028F000C157F501C158F502C159F503C1DA
:100D10005AF5006793EF06F0016793EF06F002675C
:100D200093EF06F00367D5EF06F053C557F554C5AA
:100D300058F555C559F556C55AF50F88D5EF06F043
:100D400005013067A6EF06F0D5EF06F00FBEBBEF4A
:100D500006F010A0C0EF06F001014767B7EF06F0FC
:100D60004867B7EF06F04967B7EF06F04A67BBEF91
:100D700006F0C0EF06F007AEC0EF06F0D2EF06F0C7
:100D80000501312FD5EF06F03C0E316F302FD5EF36
:100D900006F00101000E626FE00E636FA50E646F36
:100DA000010E656F0501306B0F880501626B33B76B
:100DB000DBEF06F062810CC100F10DC101F10EC143
:100DC00002F10FC103F110C104F111C105F112C10B
:100DD00006F113C107F114C108F115C109F116C1DB
:100DE0000AF117C10BF135C134F100C10CF101C199
:100DF0000DF102C10EF103C10FF104C110F105C1E3
:100E000011F106C112F107C113F108C114F109C1B2
:100E100015F10AC116F10BC117F134C135F1010109
:100E20008A671AEF07F08B671AEF07F08C671AEFE3
:100E300007F08D671EEF07F04EEF07F08EC100F14F
:100E40008FC101F190C102F191C103F10101010EC5
:100E5000046F000E056F000E066F000E076F9CEC0E
:100E600028F000C18EF101C18FF102C190F103C1E0
:100E700091F1006743EF07F0016743EF07F0026766
:100E800043EF07F003674EEF07F08AC18EF18BC185
:100E90008FF18CC190F18DC191F10F80D57ED5BEBF
:100EA00069D0D6CF47F1D7CF48F145C149F1E86ABB
:100EB000E8CF4AF1109047C100F148C101F149C1A2
:100EC00002F14AC103F101010A0E046F000E056F21
:100ED000000E066F000E076F9CEC28F003AF108029
:100EE000010154A780EF07F00F9A0F9C0F9E01019C
:100EF000000E5E6F600E5F6F3D0E606F080E616FDB
:100F0000010147BF90EF07F0486790EF07F049678E
:100F100090EF07F04A6790EF07F0F288B5EF07F01F
:100F2000F2985E6B5F6B606B616B966B976B986B07
:100F3000996B9A6B9B6B9C6B9D6B9E6B9F6BA06B75
:100F4000A16BA26BA36BA46BA56BA66BA76BA86B25
:100F5000A96BAA6BAB6BAC6BAD6BAE6BAF6BB06BD5
:100F6000B16BB26BB36BB46BB56BD76AD66A010168
:100F7000456B466B0CC100F10DC101F10EC102F1D0
:100F80000FC103F110C104F111C105F112C106F145
:100F900013C107F114C108F115C109F116C10AF115
:100FA00017C10BF135C134F1D6EF07F002C0E0FFF5
:100FB000005001C0D8FF1000A6B2DCEF07F00CC053
:100FC000A9FF0BC0A8FFA69EA69CA684F29E550E64
:100FD000A76EAA0EA76EA682F28EA694A6B2EEEF18
:100FE00007F00C2A1200A96EA69EA69CA680A85007
:100FF0000C2A120004012C0E826F17EC0BF097ECF8
:1010000029F00C50F3EC07F0E8CF00F10C50F3ECB2
:1010100007F0E8CF01F101AF13EF08F00101FF0E77
:10102000026FFF0E036F3AEC29F029671FEF08F0FB
:101030000401200E826F17EC0BF024EF08F004017E
:101040002D0E826F17EC0BF064EC27F01200076A8C
:101050000F6A106A0F010D0EC16E860EC06E030E70
:10106000C26E0F01680E896E130E926E080E8A6EA4
:101070008A6AF30E936E8B6A900E946EF18EF19ED7
:101080000E6A01015B6B5C6B5D6B576B586BF29A80
:101090000101476B486B496B4A6B4B6B4C6B4D6B5B
:1010A0004E6B4F6B506B516B526B456B466BD76AF7
:1010B000D66A0F01280ED56EF28A9D90B00ECD6EC5
:1010C00001015E6B5F6B606B616B626B636B646B8A
:1010D000656B666B676B686B696B536B546BCF6A40
:1010E000CE6A0F9A0F9C0F9E9D80760ECA6E9D82CF
:1010F00002013C0E006FCC6A160EF3EC07F0E8CF4D
:1011000000F1170EF3EC07F0E8CF01F1180EF3EC45
:1011100007F0E8CF02F1190EF3EC07F0E8CF03F186
:10112000010103AFAEEF08F097EC29F0160E0C6E3C
:1011300000C10BF0DCEC07F0170E0C6E01C10BF0D8
:10114000DCEC07F0180E0C6E02C10BF0DCEC07F0C3
:10115000190E0C6E03C10BF0DCEC07F000C18AF134
:1011600001C18BF102C18CF103C18DF100C18EF17F
:1011700001C18FF102C190F103C191F11A0EF3EC9C
:1011800007F0E8CF00F11B0EF3EC07F0E8CF01F118
:101190001C0EF3EC07F0E8CF02F11D0EF3EC07F0A4
:1011A000E8CF03F1010103AF04EF09F097EC29F058
:1011B0001A0E0C6E00C10BF0DCEC07F01B0E0C6E6F
:1011C00001C10BF0DCEC07F01C0E0C6E02C10BF041
:1011D000DCEC07F01D0E0C6E03C10BF0DCEC07F02D
:1011E0001A0EF3EC07F0E8CF00F11B0EF3EC07F05A
:1011F000E8CF01F11C0EF3EC07F0E8CF02F11D0E71
:10120000F3EC07F0E8CF03F100C192F101C193F1D3
:1012100002C194F103C195F1240EAC6E900EAB6E39
:10122000240EAC6E080EB86E000EB06E1F0EAF6EC0
:101230000401806B816B0F01900EAB6E0F019D8AD4
:101240000301806B816BC26B8B9226EC30F026EC35
:1012500030F0880EF3EC07F0E8CF00F1890EF3ECE4
:1012600007F0E8CF01F1010101AF4FEF09F097EC72
:1012700029F0880E0C6E00C10BF0DCEC07F0890E33
:101280000C6E01C10BF0DCEC07F0880EF3EC07F0FC
:10129000E8CF00F1890EF3EC07F0E8CF01F100C1CF
:1012A00040F601C141F602C142F603C143F67EECAD
:1012B00033F007EC2EF0200EF3EC07F0E8CF2FF51B
:1012C00005012F51FF0AD8A46DEF09F02F6B200EF6
:1012D0000C6E2FC50BF0DCEC07F00501010E306F32
:1012E0003C0E316F250EF3EC07F0E8CF00F1260E2F
:1012F000F3EC07F0E8CF01F1270EF3EC07F0E8CFAD
:1013000002F1280EF3EC07F0E8CF03F1010103AF7F
:10131000A4EF09F097EC29F0250E0C6E00C10BF03C
:10132000DCEC07F0260E0C6E01C10BF0DCEC07F0D4
:10133000270E0C6E02C10BF0DCEC07F0280E0C6ED1
:1013400003C10BF0DCEC07F000C153F501C154F50B
:1013500002C155F503C156F500C157F501C158F555
:1013600002C159F503C15AF5290EF3EC07F0E8CF95
:101370005BF505015C515B5DD8A05BC55CF50501C3
:101380002F51020A0EE181B8D1EF09F005015C2F5F
:10139000CEEF09F05BC55CF5D1EF09F081BABDEF86
:1013A00033F0210EF3EC07F0E8CF00F1220EF3EC5E
:1013B00007F0E8CF01F1230EF3EC07F0E8CF02F1DC
:1013C000240EF3EC07F0E8CF03F1010103AF17EFB0
:1013D0000AF097EC29F0210E0C6E00C10BF0DCEC4A
:1013E00007F0220E0C6E01C10BF0DCEC07F0230EAF
:1013F0000C6E02C10BF0DCEC07F0240E0C6E03C186
:101400000BF0DCEC07F0210EF3EC07F0E8CF00F175
:10141000220EF3EC07F0E8CF01F1230EF3EC07F016
:10142000E8CF02F1240EF3EC07F0E8CF03F100C19E
:101430005DF501C15EF502C15FF503C160F53EECEB
:101440002DF000EC2CF050EC2BF005012F51030A8D
:1014500012E005012F51040A1DE005012F51050A74
:1014600024E005012F51060A32E005012F51070A39
:1014700038E07AEF0AF0ACC500F101010F0E001759
:1014800001010051000A36E001010051050A32E075
:1014900077EF0AF0ACC500F101010F0E0017010152
:1014A0000051000A27E077EF0AF00501AC51000A6D
:1014B00021E00501AC51150A1DE00501AC51300ACF
:1014C00019E00501AC51450A15E077EF0AF0050176
:1014D000AC51000A0FE00501AC51300A0BE077EF88
:1014E0000AF00501AC51000A05E077EF0AF081BA75
:1014F000BDEF33F0FBEC2AF007900001F28EF28C86
:1015000007B0F8EF24F00FB0D9EF1FF00FB89DEF40
:1015100019F00301805181197F0BD8B4F8EF24F042
:1015200013EE00F081517F0BE126812BE7CFE8FF1E
:10153000E00BD8B4F8EF24F023EE82F0C2513F0B59
:10154000D926E7CFDFFFC22BDF50780AD8A4F8EF07
:1015500024F007808EC100F18FC101F190C102F12A
:1015600091C103F10101040E046F000E056F000E1E
:10157000066F000E076F9CEC28F000AFC9EF0AF071
:101580000101030E8E6F000E8F6F000E906F000E24
:10159000916F03018251720AD8B4D9EF1FF08251C2
:1015A000520AD8B4D9EF1FF08251750AD8B4D9EFD6
:1015B0001FF08251630AD8B4B4EF21F08251690A56
:1015C000D8B494EF1CF082517A0AD8B4A7EF1DF07A
:1015D0008251490AD8B433EF1CF08251500AD8B472
:1015E00051EF1BF08251700AD8B494EF1BF0825176
:1015F000540AD8B4BFEF1BF08251740AD8B405EF77
:101600001CF08251730AD8B409EF1FF08251530ABB
:10161000D8B46EEF1FF082514C0AD8B4FFEF11F02E
:101620008251760AD8B42BEF0BF0E9EF21F00401D8
:1016300014EE00F080517F0BE12682C4E7FF802B7F
:10164000120004010D0E826F17EC0BF00A0E826F70
:1016500017EC0BF0120003018351300AD8B4D0EF1D
:101660000CF003018351310AD8B407EF0DF00301E8
:101670008351320AD8B4BCEF0EF003018351330A10
:10168000D8B471EF10F003018351340AD8B417EFC6
:1016900011F003018351730AD8B4B2EF0BF00301C8
:1016A0008351760AD8B4B4EF0BF003018351740A66
:1016B000D8B49FEF0BF003018351540AD8B464EF00
:1016C0000BF0D8A4E9EF21F00401760E826F17EC3D
:1016D0000BF00401540E826F17EC0BF0078400012D
:1016E000880E0C6ED8EC29F02981030184512D0A53
:1016F000D8B47DEF0BF00101299185C32FF186C38A
:1017000030F187C331F188C332F189C333F1E5EC9D
:1017100029F05CEC29F000C10BF0DCEC07F001C112
:101720000BF0DCEC07F0880EF3EC07F0E8CF40F6A6
:10173000890EF3EC07F0E8CF41F6AAEF0BF00401B5
:10174000760E826F17EC0BF00401740E826F17ECAB
:101750000BF007840001880E0C6EFAEC07F007947A
:10176000FEEF19F0B2EC0BF00401760E826F17EC6D
:101770000BF00401760E826F17EC0BF0078414EC6B
:1017800026F004012C0E826F17EC0BF00101036BA5
:10179000026B3BC601F13AC600F101AFD5EF0BF089
:1017A0000101FF0E026FFF0E036F3AEC29F029676B
:1017B000DCEF0BF0E1EF0BF004012D0E826F17EC64
:1017C0000BF02FC182F40401300E822717EC0BF0CE
:1017D00030C182F40401300E822717EC0BF031C1C6
:1017E00082F40401300E822717EC0BF032C182F430
:1017F0000401300E822717EC0BF033C182F4040190
:10180000300E822717EC0BF004012C0E826F17ECC0
:101810000BF00101036B026B3DC601F13CC600F108
:1018200001AF18EF0CF00101FF0E026FFF0E036F06
:101830003AEC29F029671FEF0CF024EF0CF00401BB
:101840002D0E826F17EC0BF02FC182F40401300EC5
:10185000822717EC0BF030C182F40401300E82278E
:1018600017EC0BF031C182F40401300E822717EC23
:101870000BF032C182F40401300E822717EC0BF01A
:1018800033C182F40401300E822717EC0BF00401FF
:101890002C0E826F17EC0BF00101036B026B3FC63D
:1018A00001F13EC600F101AF5BEF0CF00101FF0E4C
:1018B000026FFF0E036F3AEC29F0296762EF0CF01C
:1018C00067EF0CF004012D0E826F17EC0BF02FC1A7
:1018D00082F40401300E822717EC0BF030C182F441
:1018E0000401300E822717EC0BF031C182F40401A1
:1018F000300E822717EC0BF032C182F40401300E57
:10190000822717EC0BF033C182F40401300E8227DA
:1019100017EC0BF004012C0E826F17EC0BF0010199
:10192000036B026B37C601F136C600F101AF9EEFC3
:101930000CF00101FF0E026FFF0E036F3AEC29F06D
:101940002967A5EF0CF0AAEF0CF004012D0E826FB1
:1019500017EC0BF02FC182F40401300E822717EC34
:101960000BF030C182F40401300E822717EC0BF02B
:1019700031C182F40401300E822717EC0BF032C122
:1019800082F40401300E822717EC0BF033C182F48D
:101990000401300E822717EC0BF00794FEEF19F0CC
:1019A0000401760E826F17EC0BF00401300E826F8B
:1019B00017EC0BF004012C0E826F17EC0BF005EC0A
:1019C0002AF097EC29F000C600F101C601F13AECCB
:1019D00029F030C182F40401300E822717EC0BF09D
:1019E00031C182F40401300E822717EC0BF032C1B2
:1019F00082F40401300E822717EC0BF033C182F41D
:101A00000401300E822717EC0BF0FEEF19F00401F1
:101A1000760E826F17EC0BF00401310E826F17EC1B
:101A20000BF007840101036B026B02C600F103C6D1
:101A300001F101AF20EF0DF0FF0E026FFF0E036FFB
:101A40000101076B066B04C604F105C605F105AF7D
:101A50002EEF0DF0FF0E066FFF0E076FA1EC28F0C2
:101A60000101076B066B06C604F107C605F105AF59
:101A70003EEF0DF0FF0E066FFF0E076FA1EC28F092
:101A80000101076B066B08C604F109C605F105AF35
:101A90004EEF0DF0FF0E066FFF0E076FA1EC28F062
:101AA000D89001010333023301330033D890010190
:101AB000033302330133003304012C0E826F17EC21
:101AC0000BF00101036B026B01C101F100C100F1D8
:101AD00001AF70EF0DF00101FF0E026FFF0E036FFB
:101AE0003AEC29F0296777EF0DF07CEF0DF0040157
:101AF0002D0E826F17EC0BF02FC182F40401300E13
:101B0000822717EC0BF030C182F40401300E8227DB
:101B100017EC0BF031C182F40401300E822717EC70
:101B20000BF032C182F40401300E822717EC0BF067
:101B300033C182F40401300E822717EC0BF001014F
:101B4000036B026B0AC600F10BC601F101AFADEFEA
:101B50000DF0FF0E026FFF0E036F0101076B066BA6
:101B60000CC604F10DC605F105AFBBEF0DF0FF0E7D
:101B7000066FFF0E076FA1EC28F00101076B066BE3
:101B80000EC604F10FC605F105AFCBEF0DF0FF0E49
:101B9000066FFF0E076FA1EC28F00101076B066BC3
:101BA00010C604F111C605F105AFDBEF0DF0FF0E15
:101BB000066FFF0E076FA1EC28F0D89001010333E8
:101BC000023301330033D890010103330233013370
:101BD000003304012C0E826F17EC0BF00101036B34
:101BE000026B01C101F100C100F101AFFDEF0DF089
:101BF0000101FF0E026FFF0E036F3AEC29F0296717
:101C000004EF0EF009EF0EF004012D0E826F17ECB9
:101C10000BF02FC182F40401300E822717EC0BF079
:101C200030C182F40401300E822717EC0BF031C171
:101C300082F40401300E822717EC0BF032C182F4DB
:101C40000401300E822717EC0BF033C182F404013B
:101C5000300E822717EC0BF00101036B026B12C6EA
:101C600000F113C601F101AF3AEF0EF0FF0E026F63
:101C7000FF0E036F0101076B066B14C604F115C656
:101C800005F105AF48EF0EF0FF0E066FFF0E076F70
:101C9000A1EC28F00101076B066B16C604F117C60C
:101CA00005F105AF58EF0EF0FF0E066FFF0E076F40
:101CB000A1EC28F00101076B066B18C604F119C6E8
:101CC00005F105AF68EF0EF0FF0E066FFF0E076F10
:101CD000A1EC28F0D8900101033302330133003323
:101CE000D8900101033302330133003304012C0E79
:101CF000826F17EC0BF00101036B026B01C101F164
:101D000000C100F101AF8AEF0EF00101FF0E026F7A
:101D1000FF0E036F3AEC29F0296791EF0EF096EF72
:101D20000EF004012D0E826F17EC0BF02FC182F420
:101D30000401300E822717EC0BF030C182F404014D
:101D4000300E822717EC0BF031C182F40401300E03
:101D5000822717EC0BF032C182F40401300E822787
:101D600017EC0BF033C182F40401300E822717EC1C
:101D70000BF00794FEEF19F00401760E826F17EC5A
:101D80000BF00401320E826F17EC0BF00784010197
:101D9000036B026B1AC600F11BC601F101AFD5EF50
:101DA0000EF0FF0E026FFF0E036F0101076B066B53
:101DB0001CC604F11DC605F105AFE3EF0EF0FF0EE2
:101DC000066FFF0E076FA1EC28F00101076B066B91
:101DD0001EC604F11FC605F105AFF3EF0EF0FF0EAE
:101DE000066FFF0E076FA1EC28F00101076B066B71
:101DF00020C604F121C605F105AF03EF0FF0FF0E79
:101E0000066FFF0E076FA1EC28F0D8900101033395
:101E1000023301330033D89001010333023301331D
:101E2000003304012C0E826F17EC0BF00101036BE1
:101E3000026B01C101F100C100F101AF25EF0FF00C
:101E40000101FF0E026FFF0E036F3AEC29F02967C4
:101E50002CEF0FF031EF0FF004012D0E826F17EC15
:101E60000BF02FC182F40401300E822717EC0BF027
:101E700030C182F40401300E822717EC0BF031C11F
:101E800082F40401300E822717EC0BF032C182F489
:101E90000401300E822717EC0BF033C182F40401E9
:101EA000300E822717EC0BF00101036B026B22C688
:101EB00000F123C601F101AF62EF0FF0FF0E026FD8
:101EC000FF0E036F0101076B066B24C604F125C6E4
:101ED00005F105AF70EF0FF0FF0E066FFF0E076FF5
:101EE000A1EC28F00101076B066B26C604F127C69A
:101EF00005F105AF80EF0FF0FF0E066FFF0E076FC5
:101F0000A1EC28F00101076B066B28C604F129C675
:101F100005F105AF90EF0FF0FF0E066FFF0E076F94
:101F2000A1EC28F0D89001010333023301330033D0
:101F3000D8900101033302330133003304012C0E26
:101F4000826F17EC0BF00101036B026B01C101F111
:101F500000C100F101AFB2EF0FF00101FF0E026FFF
:101F6000FF0E036F3AEC29F02967B9EF0FF0BEEFCF
:101F70000FF004012D0E826F17EC0BF02FC182F4CD
:101F80000401300E822717EC0BF030C182F40401FB
:101F9000300E822717EC0BF031C182F40401300EB1
:101FA000822717EC0BF032C182F40401300E822735
:101FB00017EC0BF033C182F40401300E822717ECCA
:101FC0000BF00101036B026B2AC600F12BC601F175
:101FD00001AFEFEF0FF0FF0E026FFF0E036F010175
:101FE000076B066B2CC604F12DC605F105AFFDEF9E
:101FF0000FF0FF0E066FFF0E076FA1EC28F0010136
:10200000076B066B2EC604F12FC605F105AF0DEF69
:1020100010F0FF0E066FFF0E076FA1EC28F0010114
:10202000076B066B30C604F131C605F105AF1DEF35
:1020300010F0FF0E066FFF0E076FA1EC28F0D8908E
:1020400001010333023301330033D890010103331C
:1020500002330133003304012C0E826F17EC0BF0B6
:102060000101036B026B01C101F100C100F101AF7D
:102070003FEF10F00101FF0E026FFF0E036F3AEC0D
:1020800029F0296746EF10F04BEF10F004012D0EF8
:10209000826F17EC0BF02FC182F40401300E8227FF
:1020A00017EC0BF030C182F40401300E822717ECDC
:1020B0000BF031C182F40401300E822717EC0BF0D3
:1020C00032C182F40401300E822717EC0BF033C1C9
:1020D00082F40401300E822717EC0BF00794FEEF18
:1020E00019F00401760E826F17EC0BF00401330E29
:1020F000826F17EC0BF004012C0E826F17EC0BF0C3
:1021000085C382F417EC0BF0640E0D6E030185514C
:10211000320A02E16A0E0D6E03018551330A02E1B3
:10212000700E0D6E03018551340A02E1760E0D6EBC
:1021300003018551350A02E17C0E0D6E03018551C4
:10214000360A02E1820E0D6E03018651780A65E0BF
:102150000DC00CF0D8EC29F02981030187512D0A1C
:10216000D8B4B5EF10F00101299188C32FF189C3CC
:1021700030F18AC331F18BC332F18CC333F1E5EC1A
:1021800029F05CEC29F000C10BF0DCEC07F001C198
:102190000BF0DCEC07F0D8EC29F0298103018E511B
:1021A0002D0AD8B4D6EF10F0010129918FC32FF179
:1021B00090C330F191C331F192C332F193C333F143
:1021C000E5EC29F05CEC29F000C10BF0DCEC07F049
:1021D00001C10BF0DCEC07F0D8EC29F029810301F8
:1021E00095512D0AD8B4F7EF10F00101299196C34B
:1021F0002FF197C330F198C331F199C332F19AC3EB
:1022000033F1E5EC29F05CEC29F000C10BF0DCECDB
:1022100007F001C10BF0DCEC07F00DC00CF0FAEC9C
:1022200007F0FAEC07F0FAEC07F0FEEF19F0040102
:10223000760E826F17EC0BF00401340E826F17ECF0
:102240000BF003018451780AD8B4EFEF11F03E0E81
:102250000C6ED8EC29F02981030185512D0AD8B4E0
:1022600034EF11F00101299186C32FF187C330F1BA
:1022700088C331F189C332F18AC333F1E5EC29F027
:102280005CEC29F000C10BF0DCEC07F001C10BF0B5
:10229000DCEC07F0D8EC29F0298103018C512D0AE0
:1022A000D8B455EF11F0010129918DC32FF18EC3E0
:1022B00030F18FC331F190C332F191C333F1E5ECCA
:1022C00029F05CEC29F000C10BF0DCEC07F001C157
:1022D0000BF0DCEC07F0D8EC29F0298103019351D5
:1022E0002D0AD8B476EF11F00101299194C32FF192
:1022F00095C330F196C331F197C332F198C333F1EE
:10230000E5EC29F05CEC29F000C10BF0DCEC07F007
:1023100001C10BF0DCEC07F0D8EC29F029810301B6
:102320009A512D0AD8B497EF11F0010129919BC35E
:102330002FF19CC330F19DC331F19EC332F19FC395
:1023400033F1E5EC29F05CEC29F000C10BF0DCEC9A
:1023500007F001C10BF0DCEC07F0D8EC29F0298183
:102360000301A1512D0AD8B4B8EF11F00101299150
:10237000A2C32FF1A3C330F1A4C331F1A5C332F13D
:10238000A6C333F1E5EC29F05CEC29F000C10BF0B9
:10239000DCEC07F001C10BF0DCEC07F0D8EC29F025
:1023A00029810301A8512D0AD8B4D9EF11F00101F8
:1023B0002991A9C32FF1AAC330F1ABC331F1ACC34A
:1023C00032F1ADC333F1E5EC29F05CEC29F000C14A
:1023D0000BF0DCEC07F001C10BF0DCEC07F03E0E7B
:1023E0000C6EFAEC07F0FAEC07F0FAEC07F0FAECF6
:1023F00007F0FAEC07F0FAEC07F0FEEF19F0030132
:102400008351300AD8B4C0EF14F003018351310A6C
:10241000D8B4CEEF15F003018351320AD8B43CEFA3
:1024200016F003018351330AD8B44CEF16F00301C0
:102430008351340AD8B45CEF16F003018351350A96
:10244000D8B4A2EF19F003018351360AD8B4D0EF03
:1024500019F003018351460AD8B4F6EF18F00301CE
:1024600083514D0AD8B439EF13F0030183516D0A3B
:10247000D8B453EF13F0030183515A0AD8B448EF8C
:1024800015F003018351490AD8B4D0EF1AF00301C3
:102490008351500AD8B402EF1AF003018351540A51
:1024A000D8B47BEF1AF003018351630AD8B473EFF9
:1024B00013F003018351430AD8B46BEF14F0030106
:1024C0008351730AD8B471EF13F003018351610A89
:1024D000D8B486EF12F003018351650AD8B410EF27
:1024E00015F003018351450AD8B41EEF15F003011E
:1024F0008351620AD8B42CEF15F003018351420ACC
:10250000D8B43AEF15F0D8A4E9EF21F004014C0E4D
:10251000826F17EC0BF00401610E826F17EC0BF069
:1025200000EC2CF004012C0E826F17EC0BF097ECF2
:1025300029F0ABC500F101013AEC29F031C182F478
:102540000401300E822717EC0BF032C182F4040133
:10255000300E822717EC0BF033C182F40401300EE9
:10256000822717EC0BF004012C0E826F17EC0BF096
:1025700097EC29F0ACC500F101013AEC29F031C12A
:1025800082F40401300E822717EC0BF032C182F482
:102590000401300E822717EC0BF033C182F40401E2
:1025A000300E822717EC0BF004012C0E826F17EC13
:1025B0000BF097EC29F0ADC500F101013AEC29F0E0
:1025C00031C182F40401300E822717EC0BF032C1C6
:1025D00082F40401300E822717EC0BF033C182F431
:1025E0000401300E822717EC0BF004012C0E826FD1
:1025F00017EC0BF097EC29F0AEC500F101013AECB5
:1026000029F031C182F40401300E822717EC0BF05F
:1026100032C182F40401300E822717EC0BF033C173
:1026200082F40401300E822717EC0BF004012C0E0B
:10263000826F17EC0BF097EC29F0B3C500F10101A4
:102640003AEC29F031C182F40401300E822717ECF4
:102650000BF032C182F40401300E822717EC0BF02C
:1026600033C182F40401300E822717EC0BF0FEEF29
:1026700019F0D8EC29F084C333F1E5EC29F05CECD7
:1026800029F0200E0C6E00C10BF0DCEC07F000C14D
:102690002FF505012F51000A06E005012F51010A0F
:1026A00002E0A6EC2CF004014C0E826F17EC0BF04C
:1026B00004014D0E826F17EC0BF004012C0E826F9B
:1026C00017EC0BF097EC29F02FC500F13AEC29F04C
:1026D00033C182F40401300E822717EC0BF0FEEFB9
:1026E00019F0BDEF33F004014C0E826F17EC0BF0C4
:1026F0000401630E826F17EC0BF050EC2BF0040119
:102700002C0E826F17EC0BF088EC13F0FEEF19F033
:1027100097EC29F0B1C500F10101003B0F0E001745
:102720003AEC29F033C182F40401300E822717EC11
:102730000BF0B1C500F101010F0E010100173AECD9
:1027400029F033C182F40401300E822717EC0BF01C
:1027500004012D0E826F17EC0BF0B0C500F10101E2
:10276000003B0F0E00173AEC29F033C182F404014C
:10277000300E822717EC0BF0B0C500F101010F0EEF
:10278000010100173AEC29F033C182F40401300E44
:10279000822717EC0BF004012D0E826F17EC0BF063
:1027A000AFC500F10101003B0F0E00173AEC29F014
:1027B00033C182F40401300E822717EC0BF0AFC551
:1027C00000F101010F0E010100173AEC29F033C1AD
:1027D00082F40401300E822717EC0BF00401200E66
:1027E000826F17EC0BF0AEC500F10F0E0101001760
:1027F0003AEC29F033C182F40401300E822717EC41
:102800000BF00401200E826F17EC0BF0ADC500F148
:1028100001010101003B0F0E00173AEC29F033C112
:1028200082F40401300E822717EC0BF0ADC500F1E5
:1028300001010F0E010100173AEC29F033C182F4B7
:102840000401300E822717EC0BF004013A0E826F60
:1028500017EC0BF0ACC500F10101003B0F0E0017A7
:102860003AEC29F033C182F40401300E822717ECD0
:102870000BF0ACC500F101010F0E010100173AEC9D
:1028800029F033C182F40401300E822717EC0BF0DB
:1028900004013A0E826F17EC0BF0ABC500F1010199
:1028A000003B0F0E00173AEC29F033C182F404010B
:1028B000300E822717EC0BF0ABC500F101010F0EB3
:1028C00000173AEC29F033C182F40401300E82275C
:1028D00017EC0BF0120084C3E8FF0F0BE83AE8CFC7
:1028E000B1F585C3E8FF0F0B0501B11387C3E8FFFE
:1028F0000F0BE83AE8CFB0F588C3E8FF0F0B0501EE
:10290000B0138AC3E8FF0F0BE83AE8CFAFF58BC3EB
:10291000E8FF0F0B0501AF138DC3E8FF0F0BE8CFE6
:10292000AEF58FC3E8FF0F0BE83AE8CFADF590C3E3
:10293000E8FF0F0B0501AD1392C3E8FF0F0BE83A58
:10294000E8CFACF593C3E8FF0F0B0501AC1395C3BB
:10295000E8FF0F0BE83AE8CFABF596C3E8FF0F0BA3
:102960000501AB13AFEC2BF004014C0E826F17EC9A
:102970000BF00401430E826F17EC0BF07DEF13F0A8
:1029800007847EEC33F097EC29F02DC500F13AEC8A
:1029900029F004014C0E826F17EC0BF00401300E8D
:1029A000826F17EC0BF004012C0E826F17EC0BF00A
:1029B00031C182F40401300E822717EC0BF032C1D2
:1029C00082F40401300E822717EC0BF033C182F43D
:1029D0000401300E822717EC0BF004012C0E826FDD
:1029E00017EC0BF097EC29F02EC500F13AEC29F02A
:1029F00031C182F40401300E822717EC0BF032C192
:102A000082F40401300E822717EC0BF033C182F4FC
:102A10000401300E822717EC0BF00794FEEF19F03B
:102A200004014C0E826F17EC0BF00401650E826FEF
:102A300017EC0BF08FEC2DF0FEEF19F004014C0EAB
:102A4000826F17EC0BF00401450E826F17EC0BF050
:102A5000ACEC2DF0FEEF19F004014C0E826F17EC78
:102A60000BF00401620E826F17EC0BF0E6EC2DF018
:102A7000FEEF19F004014C0E826F17EC0BF004010D
:102A8000420E826F17EC0BF0C9EC2DF0FEEF19F03F
:102A900004014C0E826F17EC0BF004015A0E826F8A
:102AA00017EC0BF004012C0E826F17EC0BF07EEC90
:102AB00033F097EC29F005012E51130A06E00501C9
:102AC0002E51170A0DE079EF15F00101000E006F8D
:102AD000000E016F100E026F000E036F79EF15F0FC
:102AE0000101000E006F000E016F000E026F010E5B
:102AF000036F0101200E046F000E056F000E066FBC
:102B0000000E076FCDEC28F03AEC29F02AC182F4D0
:102B10000401300E822717EC0BF02BC182F4040164
:102B2000300E822717EC0BF02CC182F40401300E1A
:102B3000822717EC0BF02DC182F40401300E82279E
:102B400017EC0BF02EC182F40401300E822717EC33
:102B50000BF02FC182F40401300E822717EC0BF02A
:102B600030C182F40401300E822717EC0BF031C122
:102B700082F40401300E822717EC0BF032C182F48C
:102B80000401300E822717EC0BF033C182F40401EC
:102B9000300E822717EC0BF0FEEF19F007840401CA
:102BA0004C0E826F17EC0BF00401310E826F17ECA4
:102BB0000BF004012C0E826F17EC0BF025C500F111
:102BC00026C501F127C502F128C503F10101200E38
:102BD000046F000E056F000E066F000E076FCDEC40
:102BE00028F03AEC29F02AC182F40401300E822741
:102BF00017EC0BF02BC182F40401300E822717EC86
:102C00000BF02CC182F40401300E822717EC0BF07C
:102C10002DC182F40401300E822717EC0BF02EC177
:102C200082F40401300E822717EC0BF02FC182F4DE
:102C30000401300E822717EC0BF030C182F404013E
:102C4000300E822717EC0BF031C182F40401300EF4
:102C5000822717EC0BF032C182F40401300E822778
:102C600017EC0BF033C182F40401300E822717EC0D
:102C70000BF00794FEEF19F0078404014C0E826FED
:102C800017EC0BF00401320E826F17EC0BF0DCEC4A
:102C90002FF00794FEEF19F0078404014C0E826FA9
:102CA00017EC0BF00401330E826F17EC0BF039ECCC
:102CB00030F00794D9EF15F0078404014C0E826FB1
:102CC00017EC0BF00401340E826F17EC0BF00401CB
:102CD0002C0E826F17EC0BF0D8EC29F084C32AF18C
:102CE00085C32BF186C32CF187C32DF188C32EF148
:102CF00089C32FF18AC330F18BC331F18CC332F118
:102D00008DC333F10101296BE5EC29F05CEC29F06E
:102D1000200E046F000E056F000E066F000E076F89
:102D2000ADEC28F000C121F501C122F502C123F567
:102D300003C124F531EC33F034C5ABF535C5ACF542
:102D400036C5ADF537C5AEF538C5AFF539C5B0F503
:102D50003AC5B1F588EC13F004012C0E826F17EC24
:102D60000BF03BC500F13CC501F13DC502F13EC58C
:102D700003F10101000E046F000E056F010E066FD6
:102D8000000E076FCDEC28F03AEC29F02967CBEF65
:102D900016F0D0EF16F004012D0E826F17EC0BF039
:102DA00030C182F40401300E822717EC0BF031C1E0
:102DB00082F40401300E822717EC0BF004012E0E72
:102DC000826F17EC0BF032C182F40401300E8227BF
:102DD00017EC0BF033C182F40401300E822717EC9C
:102DE0000BF004012C0E826F17EC0BF097EC29F01E
:102DF0003FC500F140C501F113EC23F004012C0E96
:102E0000826F17EC0BF097EC29F041C500F13AEC1A
:102E100029F031C182F40401300E822717EC0BF047
:102E200032C182F40401300E822717EC0BF033C15B
:102E300082F40401300E822717EC0BF004012C0EF3
:102E4000826F17EC0BF00101036B026B48C501F1B7
:102E500047C500F101AF32EF17F00101FF0E026F1D
:102E6000FF0E036F3AEC29F0296739EF17F03EEFB8
:102E700017F004012D0E826F17EC0BF02FC182F4B6
:102E80000401300E822717EC0BF030C182F40401EC
:102E9000300E822717EC0BF031C182F40401300EA2
:102EA000822717EC0BF032C182F40401300E822726
:102EB00017EC0BF033C182F40401300E822717ECBB
:102EC0000BF004012C0E826F17EC0BF00101036B69
:102ED000026B4AC501F149C500F101AF75EF17F06A
:102EE0000101FF0E026FFF0E036F3AEC29F0296714
:102EF0007CEF17F081EF17F004012D0E826F17ECB5
:102F00000BF02FC182F40401300E822717EC0BF076
:102F100030C182F40401300E822717EC0BF031C16E
:102F200082F40401300E822717EC0BF032C182F4D8
:102F30000401300E822717EC0BF033C182F4040138
:102F4000300E822717EC0BF004012C0E826F17EC69
:102F50000BF00101036B026B4CC501F14BC500F195
:102F600001AFB8EF17F00101FF0E026FFF0E036F04
:102F70003AEC29F02967BFEF17F0C4EF17F004010E
:102F80002D0E826F17EC0BF02FC182F40401300E6E
:102F9000822717EC0BF030C182F40401300E822737
:102FA00017EC0BF031C182F40401300E822717ECCC
:102FB0000BF032C182F40401300E822717EC0BF0C3
:102FC00033C182F40401300E822717EC0BF00401A8
:102FD0002C0E826F17EC0BF00101036B026B4EC5D8
:102FE00001F14DC500F101AFFBEF17F00101FF0E3C
:102FF000026FFF0E036F3AEC29F0296702EF18F019
:1030000007EF18F004012D0E826F17EC0BF02FC1A3
:1030100082F40401300E822717EC0BF030C182F4E9
:103020000401300E822717EC0BF031C182F4040149
:10303000300E822717EC0BF032C182F40401300EFF
:10304000822717EC0BF033C182F40401300E822783
:1030500017EC0BF004012C0E826F17EC0BF0010142
:10306000036B026B50C501F14FC500F101AF3EEF9C
:1030700018F00101FF0E026FFF0E036F3AEC29F00A
:10308000296745EF18F04AEF18F004012D0E826F02
:1030900017EC0BF02FC182F40401300E822717ECDD
:1030A0000BF030C182F40401300E822717EC0BF0D4
:1030B00031C182F40401300E822717EC0BF032C1CB
:1030C00082F40401300E822717EC0BF033C182F436
:1030D0000401300E822717EC0BF004012C0E826FD6
:1030E00017EC0BF00101036B026B52C501F151C5E6
:1030F00000F101AF81EF18F00101FF0E026FFF0E2A
:10310000036F3AEC29F0296788EF18F08DEF18F07B
:1031100004012D0E826F17EC0BF02FC182F4040115
:10312000300E822717EC0BF030C182F40401300E10
:10313000822717EC0BF031C182F40401300E822794
:1031400017EC0BF032C182F40401300E822717EC29
:103150000BF033C182F40401300E822717EC0BF020
:1031600004012C0E826F17EC0BF00101036B026B54
:1031700046C501F145C500F101AFC4EF18F00101EA
:10318000FF0E026FFF0E036F3AEC29F02967CBEFB9
:1031900018F0D0EF18F004012D0E826F17EC0BF031
:1031A0002FC182F40401300E822717EC0BF030C1DE
:1031B00082F40401300E822717EC0BF031C182F447
:1031C0000401300E822717EC0BF032C182F40401A7
:1031D000300E822717EC0BF033C182F40401300E5D
:1031E000822717EC0BF00794FEEF19F0D8EC29F0CA
:1031F00085C32AF186C32BF187C32CF188C32DF137
:1032000089C32EF18AC32FF18BC330F18CC331F106
:103210008DC332F18EC333F10101296BE5EC29F046
:103220005CEC29F00101010E046F000E056F000E29
:10323000066F000E076F9CEC28F0100E046F000E56
:10324000056F000E066F000E076FADEC28F000C191
:1032500029F501C12AF502C12BF503C12CF565EC56
:103260002FF004014C0E826F17EC0BF00401460E98
:10327000826F17EC0BF004012C0E826F17EC0BF031
:1032800025C500F126C501F127C502F128C503F1C6
:103290000101100E046F000E056F000E066F000E88
:1032A000076FCDEC28F03AEC29F02AC182F4040132
:1032B000300E822717EC0BF02BC182F40401300E84
:1032C000822717EC0BF02CC182F40401300E822708
:1032D00017EC0BF02DC182F40401300E822717EC9D
:1032E0000BF02EC182F40401300E822717EC0BF094
:1032F0002FC182F40401300E822717EC0BF030C18D
:1033000082F40401300E822717EC0BF031C182F4F5
:103310000401300E822717EC0BF032C182F4040155
:10332000300E822717EC0BF033C182F40401300E0B
:10333000822717EC0BF0FEEF19F00F9839EC30F004
:10334000E9EF21F004014C0E826F17EC0BF0040141
:10335000350E826F17EC0BF004012C0E826F17EC08
:103360000BF097EC29F00784B5C500F107943AEC0F
:1033700029F031C182F40401300E822717EC0BF0E2
:1033800032C182F40401300E822717EC0BF033C1F6
:1033900082F40401300E822717EC0BF0FEEF19F0D7
:1033A000FCEC2FF097EC29F033C500F13AEC29F052
:1033B00004014C0E826F17EC0BF00401360E826F85
:1033C00017EC0BF004012C0E826F17EC0BF031C1DF
:1033D00082F40401300E822717EC0BF032C182F424
:1033E0000401300E822717EC0BF033C182F4040184
:1033F000300E822717EC0BF0FEEF19F021EC0BF0EA
:10340000E9EF21F004014C0E826F17EC0BF0040180
:10341000500E826F17EC0BF004012C0E826F17EC2C
:103420000BF085C32AF186C32BF187C32CF188C327
:103430002DF189C32EF18AC32FF18BC330F18CC3D8
:1034400031F18DC332F18EC333F10101E5EC29F086
:103450005CEC29F003018451530A0DE0030184510F
:103460004D0A38E00401780E826F17EC0BF021EC66
:103470000BF0E9EF21F00401530E826F17EC0BF013
:10348000250E0C6E00C10BF0DCEC07F0260E0C6E66
:1034900001C10BF0DCEC07F0270E0C6E02C10BF043
:1034A000DCEC07F0280E0C6E03C10BF0DCEC07F02F
:1034B00000C153F501C154F502C155F503C156F5DC
:1034C00000C157F501C158F502C159F503C15AF5BC
:1034D000DFEF1AF004014D0E826F17EC0BF0290E8E
:1034E0000C6E00C10BF0DCEC07F000C15BF500C115
:1034F0005CF5DFEF1AF004014C0E826F17EC0BF055
:103500000401540E826F17EC0BF004012C0E826F35
:1035100017EC0BF084C32AF185C32BF186C32CF181
:1035200087C32DF188C32EF189C32FF18AC330F1EF
:103530008BC331F18DC332F18EC333F10101E5EC60
:1035400029F05CEC29F00101000E046F000E056FFC
:10355000010E066F000E076FADEC28F0210E0C6E09
:1035600000C10BF0DCEC07F0220E0C6E01C10BF079
:10357000DCEC07F0230E0C6E02C10BF0DCEC07F064
:10358000240E0C6E03C10BF0DCEC07F000C15DF5FE
:1035900001C15EF502C15FF503C160F5DFEF1AF00E
:1035A00004014C0E826F17EC0BF00401490E826F80
:1035B00017EC0BF004012C0E826F17EC0BF0250EAC
:1035C000F3EC07F0E8CF00F1260EF3EC07F0E8CFBC
:1035D00001F1270EF3EC07F0E8CF02F1280EF3EC2F
:1035E00007F0E8CF03F13AEC29F01DEC27F00401D5
:1035F000730E826F17EC0BF004012C0E826F17EC28
:103600000BF097EC29F0290EF3EC07F0E8CF00F16E
:103610003AEC29F01DEC27F00401730E826F17ECD1
:103620000BF004012C0E826F17EC0BF057C500F164
:1036300058C501F159C502F15AC503F13AEC29F018
:103640001DEC27F00401730E826F17EC0BF00401E0
:103650002C0E826F17EC0BF097EC29F05CC500F193
:103660003AEC29F01DEC27F004016D0E826F17EC87
:103670000BF004012C0E826F17EC0BF05DC500F10E
:103680005EC501F15FC502F160C503F104EC22F0F3
:1036900004012C0E826F17EC0BF021EC0BF0E9EF1C
:1036A00021F083C32AF184C32BF185C32CF186C397
:1036B0002DF187C32EF188C32FF189C330F18AC35E
:1036C00031F18BC332F18CC333F10101E5EC29F008
:1036D0005CEC29F0160E0C6E00C10BF0DCEC07F070
:1036E000170E0C6E01C10BF0DCEC07F0180E0C6E1F
:1036F00002C10BF0DCEC07F0190E0C6E03C10BF0ED
:10370000DCEC07F000C18AF101C18BF102C18CF140
:1037100003C18DF100C18EF101C18FF102C190F1A1
:1037200003C191F133EF1CF083C32AF184C32BF161
:1037300085C32CF186C32DF187C32EF188C32FF1E9
:1037400089C330F18AC331F18BC332F18CC333F1B9
:103750000101E5EC29F05CEC29F000C18AF101C11E
:103760008BF102C18CF103C18DF100C18EF101C159
:103770008FF102C190F103C191F133EF1CF083C3CB
:103780002AF184C32BF185C32CF186C32DF187C3A5
:103790002EF188C32FF189C330F18AC331F18CC374
:1037A00032F18DC333F10101E5EC29F05CEC29F035
:1037B0000101000E046F000E056F010E066F000E72
:1037C000076FADEC28F01A0E0C6E00C10BF0DCECAC
:1037D00007F01B0E0C6E01C10BF0DCEC07F01C0EA9
:1037E0000C6E02C10BF0DCEC07F01D0E0C6E03C179
:1037F0000BF0DCEC07F000C192F101C193F102C1C2
:1038000094F103C195F133EF1CF083C32AF184C313
:103810002BF185C32CF186C32DF187C32EF188C30C
:103820002FF189C330F18AC331F18CC332F18DC3DA
:1038300033F10101E5EC29F05CEC29F00101000E07
:10384000046F000E056F010E066F000E076FADECE2
:1038500028F000C192F101C193F102C194F103C1BA
:1038600095F133EF1CF0160EF3EC07F0E8CF00F102
:10387000170EF3EC07F0E8CF01F1180EF3EC07F0A8
:10388000E8CF02F1190EF3EC07F0E8CF03F13AECC0
:1038900029F01DEC27F00401730E826F17EC0BF07A
:1038A00004012C0E826F17EC0BF08AC100F18BC162
:1038B00001F18CC102F18DC103F13AEC29F01DEC4C
:1038C00027F00401730E826F17EC0BF004012C0E2D
:1038D000826F17EC0BF01A0EF3EC07F0E8CF00F153
:1038E0001B0EF3EC07F0E8CF01F11C0EF3EC07F030
:1038F000E8CF02F11D0EF3EC07F0E8CF03F104EC82
:1039000022F004012C0E826F17EC0BF092C100F133
:1039100093C101F194C102F195C103F104EC22F0CD
:1039200021EC0BF0E9EF21F00401690E826F17EC36
:103930000BF004012C0E826F17EC0BF00101040E4A
:10394000006F000E016F000E026F000E036F3AEC65
:1039500029F02CC182F40401300E822717EC0BF001
:103960002DC182F40401300E822717EC0BF02EC11A
:1039700082F40401300E822717EC0BF02FC182F481
:103980000401300E822717EC0BF030C182F40401E1
:10399000300E822717EC0BF031C182F40401300E97
:1039A000822717EC0BF032C182F40401300E82271B
:1039B00017EC0BF033C182F40401300E822717ECB0
:1039C0000BF004012C0E826F17EC0BF001010B0EB3
:1039D000006F000E016F000E026F000E036F3AECD5
:1039E00029F02CC182F40401300E822717EC0BF071
:1039F0002DC182F40401300E822717EC0BF02EC18A
:103A000082F40401300E822717EC0BF02FC182F4F0
:103A10000401300E822717EC0BF030C182F4040150
:103A2000300E822717EC0BF031C182F40401300E06
:103A3000822717EC0BF032C182F40401300E82278A
:103A400017EC0BF033C182F40401300E822717EC1F
:103A50000BF004012C0E826F17EC0BF00101200E0D
:103A6000006F000E016F000E026F000E036F3AEC44
:103A700029F02CC182F40401300E822717EC0BF0E0
:103A80002DC182F40401300E822717EC0BF02EC1F9
:103A900082F40401300E822717EC0BF02FC182F460
:103AA0000401300E822717EC0BF030C182F40401C0
:103AB000300E822717EC0BF031C182F40401300E76
:103AC000822717EC0BF032C182F40401300E8227FA
:103AD00017EC0BF033C182F40401300E822717EC8F
:103AE0000BF004012C0E826F17EC0BF0200EF86E19
:103AF000F76AF66A04010900F5CF82F417EC0BF0BF
:103B00000900F5CF82F417EC0BF00900F5CF82F431
:103B100017EC0BF00900F5CF82F417EC0BF009005D
:103B2000F5CF82F417EC0BF00900F5CF82F417EC17
:103B30000BF00900F5CF82F417EC0BF00900F5CF7C
:103B400082F417EC0BF021EC0BF0E9EF21F083513C
:103B5000630AD8A4E9EF21F08451610AD8A4E9EFFF
:103B600021F085516C0AD8A4E9EF21F08651410A71
:103B700042E08651440A1BE08651420AD8B40EEF57
:103B80001EF08651350AD8B473EF23F08651360AF9
:103B9000D8B4C8EF23F08651370AD8B431EF24F0F7
:103BA0008651380AD8B48FEF24F0E9EF21F0079856
:103BB000079A04017A0E826F17EC0BF00401780E5D
:103BC000826F17EC0BF00401640E826F17EC0BF0A0
:103BD00081A8F2EF1DF00401550E826F17EC0BF077
:103BE000F7EF1DF004014C0E826F17EC0BF021EC87
:103BF0000BF0E9EF21F00788079A04017A0E826F33
:103C000017EC0BF00401410E826F17EC0BF004016E
:103C1000610E826F17EC0BF0E8EF1DF00798078A32
:103C200004017A0E826F17EC0BF00401420E826FD2
:103C300017EC0BF00401610E826F17EC0BF0E8EF4C
:103C40001DF0010166672CEF1EF067672CEF1EF078
:103C500068672CEF1EF0696744EF1EF04F6738EF7E
:103C60001EF0506738EF1EF0516738EF1EF05267B4
:103C700044EF1EF00101000E006F000E016F000EF8
:103C8000026F000E036F12000101620E046F010E3D
:103C9000056F000E066F000E076F66C100F167C169
:103CA00001F168C102F169C103F19CEC28F003BF86
:103CB000C8EF1EF00101000E046FA80E056F550E2F
:103CC000066F020E076F66C100F167C101F168C19E
:103CD00002F169C103F166C186F167C187F168C16C
:103CE00088F169C189F19CEC28F003BF81EF1EF0D7
:103CF0000101000E866FA80E876F550E886F020EA9
:103D0000896F0E0EF3EC07F0E8CF18F10F0EF3EC0D
:103D100007F0E8CF19F1100EF3EC07F0E8CF1AF135
:103D2000110EF3EC07F0E8CF1BF1E5EC27F086C1AC
:103D300004F187C105F188C106F189C107F19CEC46
:103D400028F00782A9EC27F0E5EC27F00792A9EC10
:103D500027F086C100F187C101F188C102F189C154
:103D600003F10792A9EC27F0CC0E046FE00E056F6B
:103D7000870E066F050E076F9CEC28F000C118F146
:103D800001C119F102C11AF103C11BF100EF1FF0CB
:103D90000101800E006F1A0E016F060E026F000EF9
:103DA000036F4FC104F150C105F151C106F152C179
:103DB00007F19CEC28F003AFE1EF1EF097EC29F03F
:103DC00012000E0EF3EC07F0E8CF18F10F0EF3EC33
:103DD00007F0E8CF19F1100EF3EC07F0E8CF1AF175
:103DE000110EF3EC07F0E8CF1BF14FC100F150C109
:103DF00001F151C102F152C103F10782A9EC27F090
:103E000018C100F119C101F11AC102F11BC103F17E
:103E100012000401730E826F17EC0BF004012C0EDC
:103E2000826F17EC0BF0078462C166F163C167F122
:103E300064C168F165C169F14BC14FF14CC150F1EA
:103E40004DC151F14EC152F157C159F158C15AF10A
:103E500007942FEC1FF021EC0BF0E9EF21F066C185
:103E600000F167C101F168C102F169C103F101010B
:103E70003AEC29F01DEC27F00401630E826F17EC79
:103E80000BF004012C0E826F17EC0BF04FC100F108
:103E900050C101F151C102F152C103F101013AECEB
:103EA00029F01DEC27F00401660E826F17EC0BF071
:103EB00004012C0E826F17EC0BF097EC29F059C11E
:103EC00000F15AC101F101013AEC29F01DEC27F093
:103ED0000401740E826F17EC0BF0120010820401C3
:103EE000530E826F17EC0BF004012C0E826F17EC4F
:103EF0000BF083C32AF184C32BF185C32CF186C355
:103F00002DF187C32EF188C32FF189C330F18AC305
:103F100031F18BC332F18CC333F10101E5EC29F0AF
:103F20005CEC29F000C166F101C167F102C168F1E2
:103F300003C169F18EC32AF18FC32BF190C32CF119
:103F400091C32DF192C32EF193C32FF194C330F19D
:103F500095C331F196C332F197C333F10101E5EC1A
:103F600029F05CEC29F000C14FF101C150F102C110
:103F700051F103C152F1D8EC29F099C32FF19AC342
:103F800030F19BC331F19CC332F19DC333F1010188
:103F9000E5EC29F05CEC29F000C159F101C15AF1BE
:103FA0002FEC1FF004012C0E826F17EC0BF0E0EFEA
:103FB0001FF08251520A03E10F82E0EF1FF00F92CF
:103FC0008251750A03E11084E7EF1FF010948251CB
:103FD000550A03E11086EEEF1FF01096078410B229
:103FE0004BEF20F010A437EF20F0B6C166F1B7C157
:103FF00067F1B8C168F1B9C169F1BAC16AF1BBC171
:104000006BF1BCC16CF1BDC16DF1BEC16EF1BFC140
:104010006FF1C0C170F1C1C171F1C2C172F1C3C110
:1040200073F1C4C174F1C5C175F1C6C176F1C7C1E0
:1040300077F1C8C178F1C9C179F1CAC17AF1CBC1B0
:104040007BF1CCC17CF1CDC17DF1CEC17EF1CFC180
:104050007FF1D0C180F1D1C181F1D2C182F1D3C150
:1040600083F1D4C184F1D5C185F13FEF20F062C165
:1040700066F163C167F164C168F165C169F14BC163
:104080004FF14CC150F14DC151F14EC152F157C1E8
:1040900059F158C15AF107940FA06DEF20F00101BA
:1040A00092675AEF20F093675AEF20F094675AEF27
:1040B00020F095675EEF20F06DEF20F021EC1EF010
:1040C00092C104F193C105F194C106F195C107F1C4
:1040D0009CEC28F003BFB1EF21F021EC1EF00101B0
:1040E000000E046F000E056F010E066F000E076FC5
:1040F000CDEC28F010A484EF20F00401750E826F3F
:1041000017EC0BF089EF20F00401720E826F17ECB0
:104110000BF004012C0E826F17EC0BF03AEC29F037
:10412000296798EF20F00401200E826F9BEF20F0AA
:1041300004012D0E826F17EC0BF030C182F40401E4
:10414000300E822717EC0BF031C182F40401300EDF
:10415000822717EC0BF004012E0E826F17EC0BF088
:1041600032C182F40401300E822717EC0BF033C108
:1041700082F40401300E822717EC0BF004016D0E5F
:10418000826F17EC0BF004012C0E826F17EC0BF012
:104190004FC100F150C101F151C102F152C103F10F
:1041A00001013AEC29F01DEC27F00401480E826F62
:1041B00017EC0BF004017A0E826F17EC0BF0040180
:1041C0002C0E826F17EC0BF066C100F167C101F194
:1041D00068C102F169C103F101013AEC29F01DEC5B
:1041E00027F00401630E826F17EC0BF004012C0E14
:1041F000826F17EC0BF066C100F167C101F168C175
:1042000002F169C103F101010A0E046F000E056F8E
:10421000000E066F000E076FADEC28F0000E046F65
:10422000120E056F000E066F000E076FCDEC28F022
:104230003AEC29F02AC182F40401300E822717ECEF
:104240000BF02BC182F40401300E822717EC0BF027
:104250002CC182F40401300E822717EC0BF02DC123
:1042600082F40401300E822717EC0BF02EC182F489
:104270000401300E822717EC0BF02FC182F40401E9
:10428000300E822717EC0BF030C182F40401300E9F
:10429000822717EC0BF004012E0E826F17EC0BF047
:1042A00031C182F40401300E822717EC0BF032C1C9
:1042B00082F40401300E822717EC0BF033C182F434
:1042C0000401300E822717EC0BF00401730E826F8D
:1042D00017EC0BF004012C0E826F17EC0BF097EC2F
:1042E00029F059C100F15AC101F113EC23F00FB2CA
:1042F0007DEF21F00FA0AFEF21F004012C0E826FB3
:1043000017EC0BF0200EF86EF76AF66A040109004C
:10431000F5CF82F417EC0BF00900F5CF82F417EC1F
:104320000BF00900F5CF82F417EC0BF00900F5CF84
:1043300082F417EC0BF00900F5CF82F417EC0BF0C8
:104340000900F5CF82F417EC0BF00900F5CF82F4E9
:1043500017EC0BF00900F5CF82F417EC0BF021EC11
:104360000BF00F90E9EF21F00401630E826F17EC60
:104370000BF004012C0E826F17EC0BF0EFEC21F028
:1043800004012C0E826F17EC0BF062EC22F004019A
:104390002C0E826F17EC0BF0DEEC22F004012C0ED9
:1043A000826F17EC0BF00101F80E006FCD0E016F5C
:1043B000660E026F030E036F04EC22F004012C0E54
:1043C000826F17EC0BF0F4EC22F021EC0BF0E9EF2C
:1043D00021F00301C26B07901092F8EF24F0D890FF
:1043E0000E0EF3EC07F0E8CF00F10F0EF3EC07F040
:1043F000E8CF01F1100EF3EC07F0E8CF02F1110E57
:10440000F3EC07F0E8CF03F10101000E046F000E9A
:10441000056F010E066F000E076FCDEC28F03AEC29
:1044200029F02AC182F40401300E822717EC0BF028
:104430002BC182F40401300E822717EC0BF02CC143
:1044400082F40401300E822717EC0BF02DC182F4A8
:104450000401300E822717EC0BF02EC182F4040108
:10446000300E822717EC0BF02FC182F40401300EBE
:10447000822717EC0BF030C182F40401300E822742
:1044800017EC0BF031C182F40401300E822717ECD7
:104490000BF004012E0E826F17EC0BF032C182F488
:1044A0000401300E822717EC0BF033C182F40401B3
:1044B000300E822717EC0BF004016D0E826F17ECA3
:1044C0000BF01200120EF3EC07F0E8CF00F1130E20
:1044D000F3EC07F0E8CF01F1140EF3EC07F0E8CFAE
:1044E00002F1150EF3EC07F0E8CF03F101010A0E1B
:1044F000046F000E056F000E066F000E076FADEC27
:1045000028F0000E046F120E056F000E066F000EED
:10451000076FCDEC28F03AEC29F02AC182F40401AF
:10452000300E822717EC0BF02BC182F40401300E01
:10453000822717EC0BF02CC182F40401300E822785
:1045400017EC0BF02DC182F40401300E822717EC1A
:104550000BF02EC182F40401300E822717EC0BF011
:104560002FC182F40401300E822717EC0BF030C10A
:1045700082F40401300E822717EC0BF004012E0E9A
:10458000826F17EC0BF031C182F40401300E8227E8
:1045900017EC0BF032C182F40401300E822717ECC5
:1045A0000BF033C182F40401300E822717EC0BF0BC
:1045B0000401730E826F17EC0BF012000A0EF3EC7D
:1045C00007F0E8CF00F10B0EF3EC07F0E8CF01F1B4
:1045D0000C0EF3EC07F0E8CF02F10D0EF3EC07F050
:1045E000E8CF03F113EF23F0060EF3EC07F0E8CF6A
:1045F00000F1070EF3EC07F0E8CF01F1080EF3EC41
:1046000007F0E8CF02F1090EF3EC07F0E8CF03F171
:1046100013EF23F0010197EC29F0078457C100F153
:1046200058C101F107940101E80E046F800E056F77
:10463000000E066F000E076FADEC28F0000E046F41
:10464000040E056F000E066F000E076FCDEC28F00C
:10465000880E046F130E056F000E066F000E076FB5
:104660009CEC28F00A0E046F000E056F000E066F1A
:10467000000E076FCDEC28F03AEC29F00101296714
:1046800047EF23F00401200E826F4AEF23F004016C
:104690002D0E826F17EC0BF030C182F40401300E46
:1046A000822717EC0BF031C182F40401300E82270F
:1046B00017EC0BF032C182F40401300E822717ECA4
:1046C0000BF004012E0E826F17EC0BF033C182F455
:1046D0000401300E822717EC0BF00401430E826FA9
:1046E00017EC0BF0120087C32AF188C32BF189C3A2
:1046F0002CF18AC32DF18BC32EF18CC32FF18DC306
:1047000030F18EC331F190C332F191C333F1010125
:10471000296BE5EC29F05CEC29F00101000E046F37
:10472000000E056F010E066F000E076FADEC28F04E
:104730000E0E0C6E00C10BF0DCEC07F00F0E0C6ED1
:1047400001C10BF0DCEC07F0100E0C6E02C10BF097
:10475000DCEC07F0110E0C6E03C10BF0DCEC07F083
:1047600004017A0E826F17EC0BF004012C0E826F9D
:1047700017EC0BF00401350E826F17EC0BF00401FF
:104780002C0E826F17EC0BF0EFEC21F0F7EF1DF021
:1047900087C32AF188C32BF189C32CF18AC32DF179
:1047A0008BC32EF18CC32FF18DC330F18EC331F149
:1047B00090C332F191C333F10101296BE5EC29F08B
:1047C0005CEC29F0880E046F130E056F000E066F67
:1047D000000E076FA1EC28F0000E046F040E056FA9
:1047E000000E066F000E076FADEC28F00101E80E19
:1047F000046F800E056F000E066F000E076FCDEC84
:1048000028F00A0E0C6E00C10BF0DCEC07F00B0E6A
:104810000C6E01C10BF0DCEC07F00C0E0C6E02C14B
:104820000BF0DCEC07F00D0E0C6E03C10BF0DCECB2
:1048300007F004017A0E826F17EC0BF004012C0EC6
:10484000826F17EC0BF00401360E826F17EC0BF041
:1048500004012C0E826F17EC0BF0DEEC22F0F7EF68
:104860001DF087C32AF188C32BF189C32CF18AC3B9
:104870002DF18BC32EF18CC32FF18DC330F18FC37B
:1048800031F190C332F191C333F10101E5EC29F02C
:104890005CEC29F0000E046F120E056F000E066F1F
:1048A000000E076FADEC28F001010A0E046F000E38
:1048B000056F000E066F000E076FCDEC28F0120E8C
:1048C0000C6E00C10BF0DCEC07F0130E0C6E01C196
:1048D0000BF0DCEC07F0140E0C6E02C10BF0DCECFC
:1048E00007F0150E0C6E03C10BF0DCEC07F00401B1
:1048F0007A0E826F17EC0BF004012C0E826F17EC0E
:104900000BF00401370E826F17EC0BF004012C0E34
:10491000826F17EC0BF062EC22F0F7EF1DF087C30B
:104920002AF188C32BF189C32CF18AC32DF18BC3E3
:104930002EF18CC32FF18DC330F18EC331F190C3B2
:1049400032F191C333F10101296BE5EC29F05CEC04
:1049500029F0880E046F130E056F000E066F000E0F
:10496000076FA1EC28F0000E046F040E056F000E17
:10497000066F000E076FADEC28F00101E80E046F22
:10498000800E056F000E066F000E076FCDEC28F04D
:10499000060E0C6E00C10BF0DCEC07F0070E0C6E7F
:1049A00001C10BF0DCEC07F0080E0C6E02C10BF03D
:1049B000DCEC07F0090E0C6E03C10BF0DCEC07F029
:1049C00004017A0E826F17EC0BF004012C0E826F3B
:1049D00017EC0BF00401380E826F17EC0BF004019A
:1049E0002C0E826F17EC0BF0F4EC22F0F7EF1DF0B9
:1049F00081A8B6EF25F007A86FEF25F00101800E22
:104A0000006F1A0E016F060E026F000E036F4BC18E
:104A100004F14CC105F14DC106F14EC107F19CEC0A
:104A200028F003BFB6EF25F017EC27F04BC100F1DB
:104A30004CC101F14DC102F14EC103F10782A9EC55
:104A400027F018C104F119C105F11AC106F11BC103
:104A500007F1F80E006FCD0E016F660E026F030EA8
:104A6000036F9CEC28F00E0E0C6E00C10BF0DCEC1A
:104A700007F00F0E0C6E01C10BF0DCEC07F0100E0E
:104A80000C6E02C10BF0DCEC07F0110E0C6E03C1D2
:104A90000BF0DCEC07F00784010197EC29F057C11B
:104AA00000F158C101F107940A0E0C6E00C10BF021
:104AB000DCEC07F00B0E0C6E01C10BF0DCEC07F028
:104AC0000C0E0C6E02C10BF0DCEC07F00D0E0C6E40
:104AD00003C10BF0DCEC07F00798B6EF25F007AA4E
:104AE000B6EF25F00784010197EC29F057C100F1DA
:104AF00058C101F10794060E0C6E00C10BF0DCECFE
:104B000007F0070E0C6E01C10BF0DCEC07F0080E8D
:104B10000C6E02C10BF0DCEC07F0090E0C6E03C149
:104B20000BF0DCEC07F0078462C100F163C101F116
:104B300064C102F165C103F10794120E0C6E00C14D
:104B40000BF0DCEC07F0130E0C6E01C10BF0DCEC8B
:104B500007F0140E0C6E02C10BF0DCEC07F0150E22
:104B60000C6E03C10BF0DCEC07F0079A04018051D6
:104B700081197F0B0BE09EA809D014EE00F0815143
:104B80007F0BE126E750812B0F01AD6E05012F5100
:104B9000010A13E081AADDEF25F005012F51000A7B
:104BA0000AE00FB8DDEF25F005013067DDEF25F0F5
:104BB0000FB8DDEF25F0BDEF33F081B8F2EF25F04F
:104BC00000EC2CF005012F51020A02E0F2EF25F073
:104BD0005C2FF2EF25F05BC55CF50501010E306F2F
:104BE0003C0E316F80EF0AF006013251385D3351CF
:104BF000D8A0010F395D800BD8A403EF26F032C690
:104C000038F633C639F6120006013251365D33519B
:104C1000D8A0010F375D800BD8B413EF26F032C651
:104C200036F633C637F6120007841AC632F61BC6AC
:104C300033F61CC638F61DC639F6F4EC25F01EC650
:104C400032F61FC633F6F4EC25F020C632F621C644
:104C500033F6F4EC25F01AC632F61BC633F61CC642
:104C600036F61DC637F604EC26F01EC632F61FC611
:104C700033F604EC26F020C632F621C633F604ECF7
:104C800026F03851365F3951D8A03929375F97EC73
:104C900029F036C600F137C601F1A3EC29F000C1B6
:104CA0003AF601C13BF622C632F623C633F624C6D5
:104CB00038F625C639F6F4EC25F026C632F627C6B6
:104CC00033F6F4EC25F028C632F629C633F6F4ECB8
:104CD00025F022C632F623C633F624C636F625C69C
:104CE00037F604EC26F026C632F627C633F604EC77
:104CF00026F028C632F629C633F604EC26F03851E1
:104D0000365F3951D8A03929375F97EC29F036C67C
:104D100000F137C601F1A3EC29F000C13CF601C156
:104D20003DF62AC632F62BC633F62CC638F62DC60B
:104D300039F6F4EC25F02EC632F62FC633F6F4EC35
:104D400025F030C632F631C633F6F4EC25F02AC62B
:104D500032F62BC633F62CC636F62DC637F604ECE3
:104D600026F02EC632F62FC633F604EC26F030C6F7
:104D700032F631C633F604EC26F03851365F39513D
:104D8000D8A03929375F97EC29F036C600F137C62D
:104D900001F1A3EC29F000C13EF601C13FF63AC68D
:104DA00032F63BC633F63CC636F63DC637F604EC63
:104DB00026F03EC632F63FC633F604EC26F00794E2
:104DC000120018C100F119C101F11AC102F11BC191
:104DD00003F1000E046F000E056F010E066F000E4A
:104DE000076FCDEC28F029A10CEF27F02051D8B4A3
:104DF0000CEF27F018C100F119C101F11AC102F13D
:104E00001BC103F1000E046F000E056F0A0E066F42
:104E1000000E076FCDEC28F01200010104510013C1
:104E2000055101130651021307510313120001012A
:104E3000186B196B1A6B1B6B12002AC182F40401E8
:104E4000300E822717EC0BF02BC182F40401300ED8
:104E5000822717EC0BF02CC182F40401300E82275C
:104E600017EC0BF02DC182F40401300E822717ECF1
:104E70000BF02EC182F40401300E822717EC0BF0E8
:104E80002FC182F40401300E822717EC0BF030C1E1
:104E900082F40401300E822717EC0BF031C182F44A
:104EA0000401300E822717EC0BF032C182F40401AA
:104EB000300E822717EC0BF033C182F40401300E60
:104EC000822717EC0BF012002FC182F40401300E80
:104ED000822717EC0BF030C182F40401300E8227D8
:104EE00017EC0BF031C182F40401300E822717EC6D
:104EF0000BF032C182F40401300E822717EC0BF064
:104F000033C182F40401300E822717EC0BF012003B
:104F1000060E116E060E126E060E136E112E8EEF19
:104F200027F0122E8EEF27F0132E8EEF27F08B84B2
:104F3000020E116E020E126E020E136E112E9EEFF5
:104F400027F0122E9EEF27F0132E9EEF27F08B9462
:104F500012000101005305E1015303E1025301E195
:104F6000002B6CEC28F097EC29F03951006F3A5186
:104F7000016F420E046F4B0E056F000E066F000EA0
:104F8000076FADEC28F000C104F101C105F102C1C9
:104F900006F103C107F118C100F119C101F11AC1ED
:104FA00002F11BC103F107B2DAEF27F0A1EC28F000
:104FB000DCEF27F09CEC28F000C118F101C119F1D9
:104FC00002C11AF103C11BF1120097EC29F059C17B
:104FD00000F15AC101F1060EF3EC07F0E8CF04F13D
:104FE000070EF3EC07F0E8CF05F1080EF3EC07F03D
:104FF000E8CF06F1090EF3EC07F0E8CF07F19CECDF
:1050000028F000C124F101C125F102C126F103C13C
:1050100027F1290E046F000E056F000E066F000EBB
:10502000076FADEC28F0EE0E046F430E056F000E17
:10503000066F000E076FA1EC28F024C104F125C112
:1050400005F126C106F127C107F1ADEC28F000C13A
:105050001CF101C11DF102C11EF103C11FF1120EAD
:10506000F3EC07F0E8CF04F1130EF3EC07F0E8CF10
:1050700005F1140EF3EC07F0E8CF06F1150EF3EC92
:1050800007F0E8CF07F10D0E006F000E016F000E64
:10509000026F000E036FADEC28F0180E046F000EC7
:1050A000056F000E066F000E076FCDEC28F01CC1D7
:1050B00004F11DC105F11EC106F11FC107F1A1ECEC
:1050C00028F06A0E046F2A0E056F000E066F000EA0
:1050D000076F9CEC28F01200BF0EFA6E200E3A6F9C
:1050E000396BD8900037013702370337D8B07DEFDE
:1050F00028F03A2F72EF28F039073A070353D8B453
:1051000012000331070B80093F6F03390F0B010FAA
:10511000396F80EC5FF0406F390580EC5FF0405DE7
:10512000405F396B3F33D8B0392739333FA992EF0D
:1051300028F04051392712000101BCEC29F0D8B009
:105140001200010103510719346F7FEC29F0D89048
:105150000751031934AF800F12000101346BA3EC27
:1051600029F0D8A0B9EC29F0D8B012008EEC29F0C3
:1051700097EC29F01F0E366FCFEC29F00B35D8B025
:105180007FEC29F0D8A00335D8B01200362FBCEF41
:1051900028F034B1A6EC29F012000101346B04515F
:1051A0000511061107110008D8A0A3EC29F0D8A01A
:1051B000B9EC29F0D8B01200086B096B0A6B0B6BC5
:1051C000CFEC29F01F0E366FCFEC29F007510B5DA5
:1051D000D8A4F7EF28F006510A5DD8A4F7EF28F01D
:1051E0000551095DD8A4F7EF28F00451085DD8A057
:1051F0000AEF29F00451085F0551D8A0053D095F69
:105200000651D8A0063D0A5F0751D8A0073D0B5FA5
:10521000D8900081362FE4EF28F034B1A6EC29F0C5
:10522000346BA3EC29F0D890D3EC29F007510B5D37
:10523000D8A427EF29F006510A5DD8A427EF29F05A
:105240000551095DD8A427EF29F00451085DD8A0C5
:1052500036EF29F0003F36EF29F0013F36EF29F015
:10526000023F36EF29F0032BD8B4120034B1A6EC7C
:1052700029F012000101346BA3EC29F0D8B0120020
:10528000D8EC29F0200E366F00370137023703378C
:1052900011EE33F00A0E376FE7360A0EE75CD8B02E
:1052A000E76EE552372F4CEF29F0362F44EF29F007
:1052B00034B12981D890120001010A0E346F200EFA
:1052C000366F11EE29F03451376F0A0ED890E6523E
:1052D000D8B0E726E732372F67EF29F003330233E0
:1052E00001330033362F61EF29F0E750FF0FD8A0CC
:1052F0000335D8B0120029B1A6EC29F012000451F0
:1053000000270551D8B0053D01270651D8B0063D0C
:1053100002270751D8B0073D032712000051086F3C
:105320000151096F02510A6F03510B6F1200010105
:10533000006B016B026B036B12000101046B056BC8
:10534000066B076B12000335D8A012000351800BC7
:10535000001F011F021F031F003FB6EF29F0013F8E
:10536000B6EF29F0023FB6EF29F0032B342B0325CB
:1053700012000735D8A012000751800B041F051F2B
:10538000061F071F043FCCEF29F0053FCCEF29F0A3
:10539000063FCCEF29F0072B342B072512000037EE
:1053A000013702370337083709370A370B3712003E
:1053B0000101296B2A6B2B6B2C6B2D6B2E6B2F6BCA
:1053C000306B316B326B336B120001012A510F0BC2
:1053D0002A6F2B510F0B2B6F2C510F0B2C6F2D5154
:1053E0000F0B2D6F2E510F0B2E6F2F510F0B2F6F99
:1053F00030510F0B306F31510F0B316F32510F0B9A
:10540000326F33510F0B336F1200899C000EC76E41
:10541000200EC66E9E96C69EC50EC96EFF0E9EB627
:1054200002D0E82EFCD79E96C69E000EC96EFF0ED7
:105430009EB602D0E82EFCD7C9CF00F69E96C69E37
:10544000000EC96EFF0E9EB602D0E82EFCD7C9CF63
:1054500001F6898C1200000EC76E200EC66E899C64
:105460009E96C69EC80EC96EFF0E9EB602D0E82E4E
:10547000FCD79E96C69E000EC96EFF0E9EB602D049
:10548000E82EFCD7C9CF02F69E96C69E000EC96EC6
:10549000FF0E9EB602D0E82EFCD7C9CF03F6898C4A
:1054A000899C9E96C69ECA0EC96EFF0E9EB602D0FD
:1054B000E82EFCD79E96C69E000EC96EFF0E9EB6C5
:1054C00002D0E82EFCD7C9CF0AF69E96C69E000EE3
:1054D000C96EFF0E9EB602D0E82EFCD7C9CF0BF6E0
:1054E000898C899C9E96C69ECC0EC96EFF0E9EB678
:1054F00002D0E82EFCD79E96C69E000EC96EFF0E07
:105500009EB602D0E82EFCD7C9CF12F69E96C69E54
:10551000000EC96EFF0E9EB602D0E82EFCD7C9CF92
:1055200013F6898C1200000EC76E200EC66E899C81
:105530009E96C69EE80EC96EFF0E9EB602D0E82E5D
:10554000FCD79E96C69E000EC96EFF0E9EB602D078
:10555000E82EFCD7C9CF1AF69E96C69E000EC96EDD
:10556000FF0E9EB602D0E82EFCD7C9CF1BF6898C61
:10557000899C9E96C69EEA0EC96EFF0E9EB602D00C
:10558000E82EFCD79E96C69E000EC96EFF0E9EB6F4
:1055900002D0E82EFCD7C9CF22F69E96C69E000EFA
:1055A000C96EFF0E9EB602D0E82EFCD7C9CF23F6F7
:1055B000898C899C9E96C69EEC0EC96EFF0E9EB687
:1055C00002D0E82EFCD79E96C69E000EC96EFF0E36
:1055D0009EB602D0E82EFCD7C9CF2AF69E96C69E6C
:1055E000000EC96EFF0E9EB602D0E82EFCD7C9CFC2
:1055F0002BF6898C1200000EC76E200EC66E899C99
:105600009E96C69E240EC96EFF0E9EB602D0E82E50
:10561000FCD79E96C69EE40EC96EFF0E9EB602D0C3
:10562000E82EFCD7898C899C9E96C69E200EC96E5A
:10563000FF0E9EB602D0E82EFCD79E96C69E5F0E49
:10564000C96EFF0E9EB602D0E82EFCD7898C899CCD
:105650009E96C69E210EC96EFF0E9EB602D0E82E03
:10566000FCD79E96C69EC00EC96EFF0E9EB602D097
:10567000E82EFCD7898C899C9E96C69E260EC96E04
:10568000FF0E9EB602D0E82EFCD79E96C69E000E58
:10569000C96EFF0E9EB602D0E82EFCD7898C120090
:1056A0008984000EC76E220EC66E9E96C69E000EA0
:1056B000C96EFF0E9EB602D0E82EFCD79E96C69EFF
:1056C000000EC96EFF0E9EB602D0E82EFCD7C9CFE1
:1056D000ABF59E96C69E000EC96EFF0E9EB602D01A
:1056E000E82EFCD7C9CFACF59E96C69E000EC96EBB
:1056F000FF0E9EB602D0E82EFCD7C9CFADF59E9620
:10570000C69E000EC96EFF0E9EB602D0E82EFCD7D4
:10571000C9CFAEF59E96C69E000EC96EFF0E9EB610
:1057200002D0E82EFCD7C9CFAFF59E96C69E000EDC
:10573000C96EFF0E9EB602D0E82EFCD7C9CFB0F5D9
:105740009E96C69E000EC96EFF0E9EB602D0E82E33
:10575000FCD7C9CFB1F5899403EC2EF012008984EF
:10576000000EC76E220EC66E9E96C69E800EC96E35
:10577000FF0E9EB602D0E82EFCD79E96C69EABC505
:10578000C9FFFF0E9EB602D0E82EFCD79E96C69E9D
:10579000ACC5C9FFFF0E9EB602D0E82EFCD79E9680
:1057A000C69EADC5C9FFFF0E9EB602D0E82EFCD73F
:1057B0009E96C69EAEC5C9FFFF0E9EB602D0E82ECD
:1057C000FCD79E96C69EAFC5C9FFFF0E9EB602D0FF
:1057D000E82EFCD79E96C69EB0C5C9FFFF0E9EB6AA
:1057E00002D0E82EFCD79E96C69EB1C5C9FFFF0E1B
:1057F0009EB602D0E82EFCD7899403EC2EF012005E
:105800008984000EC76E220EC66E9E96C69E070E37
:10581000C96EFF0E9EB602D0E82EFCD79E96C69E9D
:10582000000EC96EFF0E9EB602D0E82EFCD7C9CF7F
:10583000ABF59E96C69E000EC96EFF0E9EB602D0B8
:10584000E82EFCD7C9CFACF59E96C69E000EC96E59
:10585000FF0E9EB602D0E82EFCD7C9CFADF59E96BE
:10586000C69E000EC96EFF0E9EB602D0E82EFCD773
:10587000C9CFAEF5899403EC2EF08984000EC76E73
:10588000220EC66E9E96C69E0F0EC96EFF0E9EB667
:1058900002D0E82EFCD79E96C69E000EC96EFF0E63
:1058A0009EB602D0E82EFCD7C9CFB3F5899403EC9D
:1058B0002EF012008984000EC76E220EC66E9E96D0
:1058C000C69E870EC96EFF0E9EB602D0E82EFCD78C
:1058D0009E96C69EABC5C9FFFF0E9EB602D0E82EAF
:1058E000FCD79E96C69EACC5C9FFFF0E9EB602D0E1
:1058F000E82EFCD79E96C69EADC5C9FFFF0E9EB68C
:1059000002D0E82EFCD79E96C69EAEC5C9FFFF0EFC
:105910009EB602D0E82EFCD7899403EC2EF0898441
:105920009E96C69E8F0EC96EFF0E9EB602D0E82EC2
:10593000FCD79E96C69EB3C5C9FFFF0E9EB602D089
:10594000E82EFCD7899403EC2EF012008984000E17
:10595000C76E220EC66E9E96C69E870EC96EFF0E3D
:105960009EB602D0E82EFCD79E96C69E000EC96E4B
:10597000FF0E9EB602D0E82EFCD79E96C69E800EE5
:10598000C96EFF0E9EB602D0E82EFCD79E96C69E2C
:10599000800EC96EFF0E9EB602D0E82EFCD79E96F2
:1059A000C69E800EC96EFF0E9EB602D0E82EFCD7B2
:1059B000899403EC2EF089849E96C69E8F0EC96E44
:1059C000FF0E9EB602D0E82EFCD79E96C69E010E14
:1059D000C96EFF0E9EB602D0E82EFCD7899403EC68
:1059E0002EF012008984000EC76E220EC66E9E969F
:1059F000C69E870EC96EFF0E9EB602D0E82EFCD75B
:105A00009E96C69E000EC96EFF0E9EB602D0E82E70
:105A1000FCD79E96C69E000EC96EFF0E9EB602D0A3
:105A2000E82EFCD79E96C69E800EC96EFF0E9EB6CF
:105A300002D0E82EFCD79E96C69E800EC96EFF0E41
:105A40009EB602D0E82EFCD7899403EC2EF0898410
:105A50009E96C69E8F0EC96EFF0E9EB602D0E82E91
:105A6000FCD79E96C69E010EC96EFF0E9EB602D052
:105A7000E82EFCD7899403EC2EF012008984000EE6
:105A8000C76E220EC66E9E96C69E8F0EC96EFF0E04
:105A90009EB602D0E82EFCD703EC2EF09E96C69E52
:105AA000810EC96EFF0E9EB602D0E82EFCD78994F7
:105AB00003EC2EF08984000EC76E220EC66E9E96F1
:105AC000C69E8F0EC96EFF0E9EB602D0E82EFCD782
:105AD00003EC2EF09E96C69E010EC96EFF0E9EB67A
:105AE00002D0E82EFCD7899403EC2EF089849E9690
:105AF000C69E910EC96EFF0E9EB602D0E82EFCD750
:105B000003EC2EF09E96C69EA50EC96EFF0E9EB6A5
:105B100002D0E82EFCD7899403EC2EF01200898481
:105B2000000EC76E220EC66E9E96C69E8F0EC96E62
:105B3000FF0E9EB602D0E82EFCD703EC2EF09E9608
:105B4000C69E810EC96EFF0E9EB602D0E82EFCD70F
:105B5000899403EC2EF012008984000EC76E220E89
:105B6000C66E9E96C69E8F0EC96EFF0E9EB602D062
:105B7000E82EFCD703EC2EF09E96C69E010EC96E51
:105B8000FF0E9EB602D0E82EFCD7899403EC2EF0CF
:105B900012008984000EC76E220EC66E9E96C69EA7
:105BA000910EC96EFF0E9EB602D0E82EFCD703EC14
:105BB0002EF09E96C69EA50EC96EFF0E9EB602D012
:105BC000E82EFCD7899403EC2EF012008984000E95
:105BD000C76E220EC66E9E96C69E910EC96EFF0EB1
:105BE0009EB602D0E82EFCD703EC2EF09E96C69E01
:105BF000000EC96EFF0E9EB602D0E82EFCD7899427
:105C000003EC2EF01200050EE82EFED7120005015F
:105C1000256B266B276B286B899A400EC76E200E6A
:105C2000C66E9E96C69E030EC96EFF0E9EB602D02D
:105C3000E82EFCD79E96C69E27C5C9FFFF0E9EB6CE
:105C400002D0E82EFCD79E96C69E26C5C9FFFF0E41
:105C50009EB602D0E82EFCD79E96C69E25C5C9FFEB
:105C6000FF0E9EB602D0E82EFCD79E96C69EC95265
:105C7000FF0E9EB602D0E82EFCD7898A0F01C950CC
:105C8000FF0A01E1120005012E51130A05E005018A
:105C90002E51170A0CE012000501E00E256FFF0ED1
:105CA000266F0F0E276F000E286F60EF2EF0050194
:105CB000E00E256FFF0E266FFF0E276F000E286F78
:105CC000899A400EC76E200EC66E9E96C69E030E23
:105CD000C96EFF0E9EB602D0E82EFCD79E96C69ED9
:105CE00027C5C9FFFF0E9EB602D0E82EFCD79E96B0
:105CF000C69E26C5C9FFFF0E9EB602D0E82EFCD771
:105D00009E96C69E25C5C9FFFF0E9EB602D0E82E00
:105D1000FCD79E96C69EC952FF0E9EB602D0E82EB4
:105D2000FCD7898A0F01C950FF0A1DE005012E51D9
:105D3000130A05E005012E51170A0BE012000501B8
:105D4000000E256F000E266F100E276F000E286FB5
:105D500012000501000E256F000E266F000E276F42
:105D6000010E286F12000501256B266B276B286B2F
:105D700005012E51130A05E005012E51170A0CE00A
:105D800012000501000E216F000E226F040E236F1A
:105D9000000E246FD5EF2EF00501000E216F000ECE
:105DA000226F800E236F000E246F21C500F122C5E3
:105DB00001F123C502F124C503F125C504F126C56F
:105DC00005F127C506F128C507F10DEC27F000C144
:105DD00025F501C126F502C127F503C128F5899AE9
:105DE000400EC76E200EC66E9E96C69E030EC96EEE
:105DF000FF0E9EB602D0E82EFCD79E96C69E27C503
:105E0000C9FFFF0E9EB602D0E82EFCD79E96C69E16
:105E100026C5C9FFFF0E9EB602D0E82EFCD79E967F
:105E2000C69E25C5C9FFFF0E9EB602D0E82EFCD740
:105E30009E96C69EC952FF0E9EB602D0E82EFCD793
:105E4000898AC950FF0A08E104C125F505C126F574
:105E500006C127F507C128F5D8900501243323335F
:105E6000223321332151E00B216F21673FEF2FF0C7
:105E700022673FEF2FF023673FEF2FF02467D5EF26
:105E80002EF00501200E2527E86A2623E86A27233D
:105E9000E86A28231200E86A05012E51130A06E079
:105EA00005012E51170A0BE0020E120005012851C0
:105EB000000A03E12751F00B07E0010E1200050173
:105EC0002851000A01E0010E120029C500F12AC57F
:105ED00001F12BC502F12CC503F125C504F126C53E
:105EE00005F127C506F128C507F19CEC28F003BF92
:105EF00012004BEC2FF05FE1899A400EC76E200E26
:105F0000C66E9E96C69E060EC96EFF0E9EB602D047
:105F1000E82EFCD7898A899A9E96C69E020EC96E83
:105F2000FF0E9EB602D0E82EFCD79E96C69E27C5D1
:105F3000C9FFFF0E9EB602D0E82EFCD79E96C69EE5
:105F400026C5C9FFFF0E9EB602D0E82EFCD79E964E
:105F5000C69E25C5C9FFFF0E9EB602D0E82EFCD70F
:105F60009E96C69E000EC96EFF0E9EB602D0E82E0B
:105F7000FCD7898A899A9E96C69E050EC96EFF0E29
:105F80009EB602D0E82EFCD79E96C69EC952FF0E42
:105F90009EB602D0E82EFCD7C9B0C4EF2FF0898A94
:105FA0000501200E2527E86A2623E86A2723E86AE8
:105FB000282365EF2FF01200899A400EC76E200E3D
:105FC000C66E9E96C69E060EC96EFF0E9EB602D087
:105FD000E82EFCD7898A899A9E96C69EC70EC96EFE
:105FE000FF0E9EB602D0E82EFCD7898A0501256BEC
:105FF000266B276B286B1200899A400EC76E200E05
:10600000C66E9E96C69E050EC96EFF0E9EB602D047
:10601000E82EFCD79E96C69EC952FF0E9EB602D0B1
:10602000E82EFCD7C9CF33F5898A1200899A400E31
:10603000C76E200EC66E9E96C69EB90EC96EFF0E26
:106040009EB602D0E82EFCD7898A1200899A400EAB
:10605000C76E200EC66E9E96C69EAB0EC96EFF0E14
:106060009EB602D0E82EFCD7898AFF0EE82EFED716
:1060700012004BEC2FF0D8A41200899A400EC76E84
:10608000200EC66E9E96C69E030EC96EFF0E9EB66D
:1060900002D0E82EFCD79E96C69E27C5C9FFFF0EEC
:1060A0009EB602D0E82EFCD79E96C69E26C5C9FF96
:1060B000FF0E9EB602D0E82EFCD79E96C69E25C542
:1060C000C9FFFF0E9EB602D0E82EFCD79E96C69E54
:1060D000C952FF0E9EB602D0E82EFCD7898A0F0166
:1060E000C950FF0AD8A430EF33F00501FE0E336F1C
:1060F00050EC2BF0ABC534F5ACC535F5ADC536F578
:10610000AEC537F5AFC538F5B0C539F5B1C53AF507
:106110000784B6C166F1B7C167F1B8C168F1B9C10A
:1061200069F14BC14FF14CC150F14DC151F14EC11C
:1061300052F157C159F158C15AF121EC1EF000C17A
:106140003BF501C13CF502C13DF503C13EF505013A
:106150005D67B2EF30F05E67B2EF30F05F67B2EFCD
:1061600030F06067B6EF30F0C3EF30F05DC504F19A
:106170005EC505F15FC506F160C507F19CEC28F02E
:1061800003BF30EF33F059C13FF55AC140F5B5C5F3
:1061900041F5B6C542F514EC26F036C645F537C6CE
:1061A00046F506014067DCEF30F04167DCEF30F088
:1061B0004267DCEF30F04367E0EF30F0F1EF30F0B2
:1061C00097EC29F09DEC29F036C600F137C601F1B5
:1061D00040C604F141C605F19CEC28F003AF30EF56
:1061E00033F00101036B026B1AC600F11BC601F10B
:1061F00001AFFFEF30F0FF0E026FFF0E036F0101E2
:10620000076B066B1CC604F11DC605F105AF0DEF4B
:1062100031F0FF0E066FFF0E076FA1EC28F00101B1
:10622000076B066B1EC604F11FC605F105AF1DEF17
:1062300031F0FF0E066FFF0E076FA1EC28F0010191
:10624000076B066B20C604F121C605F105AF2DEFE3
:1062500031F0FF0E066FFF0E076FA1EC28F0D8900B
:1062600001010333023301330033D89001010333BA
:1062700002330133003300C147F501C148F5010184
:10628000036B026B22C600F123C601F101AF4DEF93
:1062900031F0FF0E026FFF0E036F0101076B066BFB
:1062A00024C604F125C605F105AF5BEF31F0FF0E02
:1062B000066FFF0E076FA1EC28F00101076B066B5C
:1062C00026C604F127C605F105AF6BEF31F0FF0ECE
:1062D000066FFF0E076FA1EC28F00101076B066B3C
:1062E00028C604F129C605F105AF7BEF31F0FF0E9A
:1062F000066FFF0E076FA1EC28F0D8900101033361
:10630000023301330033D8900101033302330133E8
:10631000003300C149F501C14AF50101036B026B6D
:106320002AC600F12BC601F101AF9BEF31F0FF0E41
:10633000026FFF0E036F0101076B066B2CC604F1A1
:106340002DC605F105AFA9EF31F0FF0E066FFF0E68
:10635000076FA1EC28F00101076B066B2EC604F154
:106360002FC605F105AFB9EF31F0FF0E066FFF0E36
:10637000076FA1EC28F00101076B066B30C604F132
:1063800031C605F105AFC9EF31F0FF0E066FFF0E04
:10639000076FA1EC28F0D8900101033302330133D9
:1063A0000033D8900101033302330133003300C1BD
:1063B0004BF501C14CF50101036B026B02C600F104
:1063C00003C601F101AFE9EF31F0FF0E026FFF0EDE
:1063D000036F0101076B066B04C604F105C605F1E6
:1063E00005AFF7EF31F0FF0E066FFF0E076FA1EC60
:1063F00028F00101076B066B06C604F107C605F11C
:1064000005AF07EF32F0FF0E066FFF0E076FA1EC2E
:1064100028F00101076B066B08C604F109C605F1F7
:1064200005AF17EF32F0FF0E066FFF0E076FA1ECFE
:1064300028F0D89001010333023301330033D890A0
:106440000101033302330133003300C14DF501C1B3
:106450004EF50101036B026B0AC600F10BC601F198
:1064600001AF37EF32F0FF0E026FFF0E036F010135
:10647000076B066B0CC604F10DC605F105AF45EFC1
:1064800032F0FF0E066FFF0E076FA1EC28F001013E
:10649000076B066B0EC604F10FC605F105AF55EF8D
:1064A00032F0FF0E066FFF0E076FA1EC28F001011E
:1064B000076B066B10C604F111C605F105AF65EF59
:1064C00032F0FF0E066FFF0E076FA1EC28F0D89098
:1064D00001010333023301330033D8900101033348
:1064E00002330133003300C14FF501C150F5010102
:1064F000036B026B12C600F113C601F101AF85EF09
:1065000032F0FF0E026FFF0E036F0101076B066B87
:1065100014C604F115C605F105AF93EF32F0FF0E76
:10652000066FFF0E076FA1EC28F00101076B066BE9
:1065300016C604F117C605F105AFA3EF32F0FF0E42
:10654000066FFF0E076FA1EC28F00101076B066BC9
:1065500018C604F119C605F105AFB3EF32F0FF0E0E
:10656000066FFF0E076FA1EC28F0D89001010333EE
:10657000023301330033D890010103330233013376
:10658000003300C151F501C152F507940501210EF8
:10659000326F899A400EC76E200EC66E9E96C69EBA
:1065A000060EC96EFF0E9EB602D0E82EFCD7898A71
:1065B000899A9E96C69E020EC96EFF0E9EB602D0A6
:1065C000E82EFCD79E96C69E27C5C9FFFF0E9EB635
:1065D00002D0E82EFCD79E96C69E26C5C9FFFF0EA8
:1065E0009EB602D0E82EFCD79E96C69E25C5C9FF52
:1065F000FF0E9EB602D0E82EFCD725EE33F0322FE8
:1066000002D00EEF33F09E96C69EDECFC9FFFF0E7E
:106610009EB602D0E82EFCD7FFEF32F0898A899A25
:106620009E96C69E050EC96EFF0E9EB602D0E82E3F
:10663000FCD79E96C69EC952FF0E9EB602D0E82E8B
:10664000FCD7C9B019EF33F0898A0501200E252740
:10665000E86A2623E86A2723E86A282388EC27F0DB
:10666000120021C500F122C501F123C502F124C5A4
:1066700003F1899A400EC76E200EC66E9E96C69E86
:106680000B0EC96EFF0E9EB602D0E82EFCD79E966A
:10669000C69E02C1C9FFFF0E9EB602D0E82EFCD7EF
:1066A0009E96C69E01C1C9FFFF0E9EB602D0E82E7F
:1066B000FCD79E96C69E00C1C9FFFF0E9EB602D0B3
:1066C000E82EFCD79E96C69EC952FF0E9EB602D0FB
:1066D000E82EFCD725EE33F00501200E326F9E9692
:1066E000C69EC952FF0E9EB602D0E82EFCD7C9CF77
:1066F000DEFF322F6FEF33F0898A1200899A400E45
:10670000C76E200EC66E9E96C69E900EC96EFF0E78
:106710009EB602D0E82EFCD79E96C69E000EC96E8D
:10672000FF0E9EB602D0E82EFCD79E96C69E000EA7
:10673000C96EFF0E9EB602D0E82EFCD79E96C69E6E
:10674000000EC96EFF0E9EB602D0E82EFCD79E96B4
:10675000C69EC952FF0E9EB602D0E82EFCD7C9CF06
:106760002DF59E96C69EC952FF0E9EB602D0E82E0B
:10677000FCD7C9CF2EF5898A120088EC27F0B5C561
:10678000E8FFD70802E388EC27F0B5C5E8FFC808A2
:1067900002E388EC27F0B5C5E8FFB90802E388EC0E
:1067A00027F0B5C5E8FFAA0802E388EC27F0B5C5D5
:1067B000E8FF9B0802E388EC27F000EC2CF016ECD5
:1067C00030F0F29CF29E8B94C69AC290898C94828F
:1067D000948C720ED36ED3A4FED789968A90939030
:1067E000FF0EE8CF00F0E82EFED7002EFCD7815038
:1067F000F294F29A9E909D909E929D92F298F292BF
:0A680000F290F286F28E0300FF0012
:10BF0000E844F926000C160C2B0C3F0C520C640C68
:10BF1000760C860C960CA50CB30CC10CCF0CDC0C6B
:06BF2000E80CF40C000C1B
:00000001FF
